:1060490047415445202D3E49533A20004741544584
:08605900202D3E52463A2000C2
:1060E9007B017A007980227B017A00790090010096
:0360F900E0FD22A5
:1058140030003BC200D211C2A1E4FF12052EEF6496
:105824000170291260E9122CACC2961260E9123799
:105834004A1260E912621D7BFF7A607949E4FD1225
:0F58440033D91260E9E4FD1233D9D296D2A122F2
:10594B00300137C201C211C2A1E4FF12052EEF6470
:10595B000170251260F01250801260F0123A47125B
:10596B0060E9122CAC7BFF7A607955E4FD1233D9D8
:0A597B001260E9E4FD1233D9D2A155
:0159850022FF
:1059F8000D0A494F31202D3E544E433A2000575846
:105A080020426F617264206E6F206C696E6B0D0AA4
:105A18000041504757314B0041504757314B0054D4
:075A2800435049502000002B
:10488600EF9325E0FF900210E02400F582E4340067
:10489600F583EFF0900210E004F022E025E044609A
:1048A600FF900210E02400F582E43400F58322EF45
:1048B600F090020FE004F02290020FE0FFC394068E
:1048C60022EFF0900212E004F022A3F0E490020F2F
:1048D600F022900211E004F02290020FE02419F574
:1048E60082E43402F5832290020FE02422F582E46A
:1048F6003402F5832290020FE024CEF582E43402DE
:10490600F583E0FF2274032FF582E43401F583E09A
:01491600227E
:10603000308315E4FFFE1260A6EF600C12581412B4
:09604000594B12574712578D22EB
:05052E0090020EEFF049
:10053300E4900210F0EF701490020FF01248BE50D6
:1005430020905A201248861248B780F0E490020F98
:10055300F01248BE500B905A191248861248B780C1
:10056300F01248A77460124899E490020FF0124801
:10057300BE50277E001260A6900218EFF07008129A
:1005830048A77440F0800B900218E025E01248A6BB
:10059300EFF012489A1248B780D490020EE070052B
:1005A3007F87FE80047F077E011260A6900217EF0B
:1005B300F0201103301229900217E025E044E012E5
:1005C300488AE490020FF01248BE500CEF905A276D
:1005D3001248871248B780EF1248A774E10206DE7B
:1005E30090020EE0900213701204F0A37490F07F57
:1005F300961209557497F07F9D80117401F0A374CE
:10060300A0F07FA612095574A7F07FAD7E0112609A
:10061300A690022AEFF0900217E025E044E012488A
:10062300A6EFF0900213120967605112489AE49002
:10063300020FF01248BE5023900214E090021312EE
:10064300094670081248DF7420F0800A900218E00F
:10065300FF1248DFEFF01248B780D8E490020FF0A2
:100663001248BE500F74192F1248E5E01248881241
:1006730048B780EC9002211248A1EFF090021512C6
:100683000967605112489AE490020FF01248BE5075
:1006930023900216E090021512094670081248EDE5
:1006A3007420F0800A900218E0FF1248EDEFF01278
:1006B30048B780D8E490020FF01248BE500F74225E
:1006C3002F1248F3E01248881248B780EC90022AB0
:1006D3001248A1EFF01248A7E044011248991248CA
:1006E300A774031248991248AA74F0124899900209
:1006F3000EE060030207AD7F88FE1260A612488BEE
:10070300A3E4F074901248D01208EE1248C77003A5
:100713001248D812489A1248B7E0C3940840E97FB8
:10072300897E001260A612488BA3E4F074A01248DD
:10073300D01208EE1248C770031248D812489A1212
:1007430048B7E0C3940940E97F8A7E001260A6128D
:10075300488BA3E4F0A374B01248D112093960178F
:100763001209071248C770031248D812489A124850
:10077300B7E0D3941F40E47F857E001260A6EF6448
:100783000160030208E01248A77420124899124737
:10079300F2E490020FF01248FB600C1248A71248D3
:1007A300B5A3E004F080EF0208E090020EE06401DC
:1007B30060030208EB7F087E011260A612488BA338
:1007C3007401F0A374101248D11209071248C770BC
:1007D300031248D812489A1248B7E0C3940840E974
:1007E3007F097E011260A612488BA37401F0A374E3
:1007F300201248D11209201248C770031248D81298
:10080300489A1248B7E0C3940940E97F0A7E01126F
:1008130060A612488BE4FF125156EF701D7BFF7ADE
:100823005979F8FD1233D97A5A79061209717A0087
:100833007980E4FD1210E87F00227A5979F81209D1
:10084300717A017903E4FD1233D990020F7401F038
:1008530090020FE0FFC39404500B12490B12488A15
:100863001248B780EB1248A7742F12489990020FD1
:100873007405F090020FE0FFC39421500B12490B53
:1008830012488A1248B780EB9002117401F0A374E6
:10089300301248D112093960171209201248C77063
:1008A300031248D812489A1248B7E0D3941F40E481
:1008B3007F057E011260A6EF640170211248A774C0
:1008C300201248991247F2E490020FF01248FB609D
:1008D3000C1248A71248B5A3E004F080EF90021071
:0A08E300E0900100F07F01227F0089
:1008ED0022900211E0FEA3E0FF1260A6900210E03C
:1008FD002400F582E43400F58322900211E0FEA37A
:10090D00E0FF1260A6900210E02400F582E43400AE
:10091D00F58322900211E0FEA3E0FF1260A6900283
:10092D0010E02400F582E43400F58322900211E0FA
:10093D00FEA3E0FF1260A6EF222FFFE03400FE12AF
:10094D0060A6900218EFF0227E011260A69002219F
:10095D00EFF09002157401F0A322E0FEA3E0FF1268
:0E096D0060A6EF227BFFE4FD1233D97B01224E
:100026000D0A575820202D3E4953203A20000D0A2C
:0C003600575820202D3E5246203A200052
:1060FC007B017A007980227B017A00790090010083
:03610C00E0FD2291
:10574700300442C204D212C2A17F0112052EEF64B7
:105757000170301260FC122CAC1260FC12374A1236
:1057670060FC12621D7BFF7A007926E4FD1233D9B3
:105777001260FCE4FD1233D97B017A0179037D01C4
:065787001210E8D2A1227D
:105DEE00900103E064636007E4900185F0FF229068
:105DFE000185E064246004E4F0FF229002F874014F
:075E0E00F0E4F5AF7F012273
:10578D00300342C203C212C2A17F0112052EEF6483
:10579D00017030126103125080126103123A4712E8
:1057AD0060FC122CAC7BFF7A007934E4FD1233D906
:1057BD001260FCE4FD1233D97B017A0179037D017E
:0657CD001210E8D2A12237
:0551560090023DEFF0A6
:10515B00E4F5AF90018404F0759CF4E4F5A29002A1
:10516B00F8F0900185F090023EF090023EE0FFC314
:10517B009480501474032FF582E43401F583E4F02A
:10518B0090023EE004F080E275AF01E490023EF045
:10519B009002F8E070177F02FE125F8D90023EE0E6
:1051AB0004F0E0D3946440E8E4F5AFFF22E4F5AFFC
:0251BB007F0172
:0151BD0022CF
:105F3300202020202020202020202020200D0A00A7
:0E5F43004750532D3E42454143454E3A200003
:105E3C00900100E0FF9002FDE0FEC39F2274002E53
:105E4C00F582E43400F583E0FF227B017A007900CF
:065E5C00900100E0FD22B0
:103F0200C2A1123FDB7F0312052E125E56125080B1
:103F1200125E56123A477FC012624BE4FF12624BA6
:103F2200E49002FDF0125E3C500E125E4912624BAA
:103F32009002FDE004F080ED7FC012624B7B017ABB
:103F4200007980122CAC7B017A00798012374A7B8F
:103F5200FF7A5F7943123FC5123FC512621D7F840B
:103F62007E011260A6EF14600E14602614604624CF
:103F7200037047E4FF8040E49002FDF09002FDE010
:103F82002480F582E43400F583E0FF602D123FD1F6
:103F920080EA7FC012608FE4FF12608FE49002FD1E
:103FA200F0125E3C5008125E49123FD180F37FC08E
:103FB20012608F80057F01121973123FDB122AE60D
:023FC200D2A18A
:103FC40022E4FD1233D97B017A0079802212608FBA
:103FD4009002FDE004F0227BFF7A5F7933E4FD1266
:033FE40033D922AC
:1044A6000D0A50494E47204641494C2C5345525619
:1044B6004552204F46464C494E45200D0A000D0AEE
:1044C600534552564552204C494E4B205354415267
:1044D600542E2E2E0D0A0053455256455220434C5B
:1044E6004F534520210D0A0053455256455220543C
:1044F60043502F4950204C494E4B204F5554544958
:104506004D45210D0A0053455256455220544350FD
:104516002F4950204C494E4B204F555454494D4538
:10452600203E2033202C4E6F7720544E4320526578
:1045360073657420210D0A00757365722000207062
:1045460061737320002056657273204757313030EF
:074556003020313038200055
:104B460090022BE02480F582E43400F58322900263
:104B56001CE0FEA3E0FF90021AE0FCA3E0FD900239
:104B660017E02DFD900216E03CFC22F090022BE0AF
:104B760004F022EFF090022AE004F0A3E004F02211
:104B86009002107404F0A3E4F0223400FEF0A3EFC8
:104B9600F0EE5407FEE42FFFEE344022FF90021C95
:104BA600E03400FE22EFF0900227E004F022340009
:104BB600F0A3CEF022900226E004F022900226E432
:034BC600F0A32237
:102E5E0090021C124B892402FFE43404FE125B8F95
:102E6E00900212EFF07D0212000EEF640160030279
:102E7E002FD390021DE02402124BA2900212E044C6
:102E8E0004FD125E6990021DE02426122FD47F00ED
:102E9E00FEC006C00790021DE02427122FD4FDD0DD
:102EAE00E02DFED0E090021A124BB490021DE024E9
:102EBE0028124BA2125B8FEF7F00FEC006C0079058
:102ECE00021DE02429124BA2125B8FEFFDD0E02DE4
:102EDE00FED0E0900216124BB4D390021BE0948009
:102EEE0090021AE094004006124B5402589290023F
:102EFE0016E05407FEA3E02400FFEE3460A3F0A317
:102F0E00EFF0A3E0FFA3E0900214CFF0A3EFF0E404
:102F1E00900213F0900214E07002A3E0604C900255
:102F2E0018E0FEA3E0FF125B8F900213124B49EFE5
:102F3E00F0900219E004F07006900218E004F09090
:102F4E000213E004F0900215E024FFF0900214E06A
:102F5E0034FFF0900218E0B468BAA3E0B400B59064
:102F6E0002187460F0A3E4F080AA900213124B4989
:102F7E00E4F0124B541258927B017A007980E4FDF2
:102F8E001233D9900080E0642370339002DEF0207B
:102F9E000A33900213F0FF900213124B49E0FE60C9
:102FAE000EB420010F900213E004F0EFB403E8908A
:102FBE000213124B49E0B47602D20A021E48C2A195
:052FCE001232A6D2A1A1
:0E2FD30022FF90021CE03400FE125B8FEF2202
:106159009002DEE004F0E0D3943C4004E4F0D20B7A
:016169002213
:105F51009002DDE0FFB4020F0512E512D394024076
:0E5F61000CE4F512B2B722EFB40302B2B7227D
:105F6F001235049002DF7413F0A37488F0751301D7
:0E5F7F00E49002DCF0A3F0F512A3F0C20B22B6
:105CC800E4FFFE1260A690020DEFF07F097E00123D
:105CD80060A620810C90020DE06006EF60030226AA
:0A5CE800F6E49002DDF0D2B7D29688
:015CF200228F
:105B00009002E0E004F070069002DFE004F0D39031
:105B100002E0E0948D9002DFE0941340137413F0E0
:105B2000A37488F00513E513D394034003751301A0
:015B30002252
:1026F600124B86300B159002DEF0C20B125B00E423
:102706009002DDF07A4479A61228EE9002DDE060B0
:10271600030228107A4479C41228EE124B86D2B7E7
:10272600C209C20A9002DEF0C20BFF1228C690024E
:10273600DFE0FD7404FFFE125E699002DFA3E0FD98
:102746007F057E04125E697F011228C61228B964CD
:102756001360030228077F2FFE1260A6EF64017044
:10276600057F22FE800DE51324FE602304703C7F66
:10277600227E001260A6AD071228CE7F231228857E
:102786001228D67F241228851228DE7F2580427FD4
:10279600261228A91228CE7F271228A91228D67F0A
:1027A600281228B11228DE7F2980267F2A1228B116
:1027B6007F0C7E04125E697F2B1228E67F0D7E0455
:1027C600125E697F2C1228E67F0E7E04125E697FF8
:1027D6002D7E001260A6AD077F0F7E04125E697D16
:1027E600387F107E04125E697DF47F117E04125ECE
:1027F600697D047F017E04125E699002DD7401F03A
:10280600227D107F017E04025E691228B9BF17136C
:102816009002DD200A057403F080057405F0C2B746
:10282600022E5E9002DD7402F0FF7E04125B8F9032
:10283600020FEFF030E10EE0440212288D7A44795F
:10284600DDFD0233D990020FE030E332440812284E
:102856008D7A4479EEFD1233D97F307E001260A660
:10286600BF011B9002DCE004F0E0D39403400FE4C8
:0E287600F07BFF7A45790CFD1233D975C7202F
:10288400227E001260A6AD0722FD7F027E04125E46
:10289400697D107F017E04125E69125B00E4900280
:1028A400DDF07BFF227E001260A6AD07227E0012BF
:1028B40060A6AD07227F037E04125B8F90020EEFA9
:1028C400F0227D017E04125E69227F0C7E04125E7A
:1028D40069227F0D7E04125E69227F0E7E04125EE1
:1028E40069227E001260A6AD07227BFFFD1233D958
:0128F40022C1
:101E4800300903022056E4FFFE1260A6EF70030279
:101E580020567F091220887003022056E490022B36
:101E6800F090022AF090022AE090453E93FF600825
:101E7800124B46124B7980EDE4900226F0A3F01243
:101E88002057EF6013122057124B46124BAB7003CA
:101E9800124BBB124B7280E77F071220886030120A
:101EA8004B46742D124B71EFC3940AEF5002801504
:101EB80075F00A842430FE124B46EE124B71EF7512
:101EC800F00A84E5F02430FF124B49EF124B71E41D
:101ED80090022AF090022AE090454493FF6008128D
:101EE8004B46124B7980ED124BC27409F0122063F5
:101EF800EF6013122063124B46124BAB7003124B68
:101F0800BB124B7280E7E490022AF090022AE0901C
:101F1800454B93FF6008124B46124B7980ED124BEC
:101F2800C27440F0FF7E001260A6EFC394FF501FFA
:101F3800124BC27440F012207CEF601312207C1206
:101F48004B46124BAB7003124BBB124B7280E7121D
:101F58004B46740D124B71124B49740A124B711295
:101F68004B49E4F0900228124B892420FFE4340402
:101F7800FE125B8FEF7F00FEC006C007900229E0CB
:101F8800242112206FFDD0E02DFED0E03400900215
:101F980020F0A3CEF0900229E0242412206F7F00C5
:101FA800FEC006C007900229E02425FF900228E021
:101FB8003400FE125B8FEFFDD0E02DFFD0E09002E1
:101FC8001E124B90900222F0A3EFF0E4A3F0A3F0CE
:101FD80090022AF090022A124B49E0FD60449002D8
:101FE80022E0FEA3E0FF125E69900223E004F07095
:101FF80006900222E004F090022AE004F090022504
:10200800E004F07006900224E004F0900222E0B4AC
:1020180048C2A3E0B400BD9002227440F0A3E4F0EB
:1020280080B2900228E0FEA3E0FF900224E0FCA327
:10203800E0FD90021FE02DFD90021EE03CFC125ACC
:0E204800667B017A007980E4FD1233D9D2095B
:1020560022900226E0FEA3E0FF1260A6229002264E
:10206600E0FEA3E0FF1260A622FF900228E0340003
:10207600FE125B8FEF22900226E0FEA3E0FF1260C5
:09208600A6227E001260A6EF22E2
:0B374A0090020FEBF0A3EAF0A3E9F0FF
:103755009002DDE06405600302384AC29690021AC1
:10376500124B892420FFE43404FE125B8FEF7F00A7
:10377500FEC006C00790021BE0242112384BFDD085
:10378500E02DFED0E03400900216F0A3CEF09002BA
:103795001BE0242412384B7F00FEC006C0079002B0
:1037A5001BE02425FF90021AE03400FE125B8FEF28
:1037B500FDD0E02DFFD0E0900214124B909002183E
:1037C500F0A3EFF0E4900212F0A3F090020FE0FBFB
:1037D500A3E0FAA3E0F9120301FD6048900218E0A6
:1037E500FEA3E0FF125E69900219E004F0700690F6
:1037F5000218E004F0900210E475F0011203D09075
:103805000213E004F07006900212E004F090021832
:10381500E0B448B7A3E0B400B29002187440F0A336
:10382500E4F080A790021AE0FEA3E0FF900212E008
:10383500FCA3E0FD900215E02DFD900214E03CFC98
:05384500125A66D29644
:0E384A0022FF90021AE03400FE125B8FEF2284
:104C4B002352455345540023494E5354414C4C0079
:104C5B0023474154455F52465F5445535400234705
:104C6B004154455F49535F54455354002357585F94
:104C7B0052465F54455354002357585F49535F5472
:104C8B00455354002348454C4C4F000D0A00632EEE
:104C9B002E2E732E2E2E672E2E2E742E2E2E722E21
:104CAB002E2E702E2E2E682E2E622E2E2E2E2E0D8A
:104CBB000A002348454C4C4F000000000000000048
:014CCB0000E8
:104BC900900212E05407FEA3E02400FFEE34709037
:104BD90002EFF0A3EFF02290022DE0FBA3E0FAA38D
:104BE900E0F902030190022DE475F0010203D034CB
:104BF90000FEF0A3EFF0EE5407FEE42FFFEE345071
:104C090022FF90022BE03400FE229002EFF0A3E491
:104C1900F022EBF0A3EAF0A3E9F0227406F0A3E492
:104C2900F02420FFE43406FE22E49002EEF0C213E1
:104C3900223400F0A3CEF0229002357450F0A3E4A0
:024C4900F02257
:0A624100208103024917124C32229B
:03628100C2132223
:1016DC00781C7C027D017BFF7A4C79BD7E007F0FEC
:1016EC001202DB90022B7406F0A3E4F02402FFE458
:1016FC003406FE125B8F900210EFF07D0212000E8A
:10170C00EF6401600302191A90022CE02402124CBF
:10171C000A900210E04404FD125E6990022CE02451
:10172C00261219577F00FEC006C00790022CE02439
:10173C0027121957FDD0E02DFED0E0900214124C68
:10174C003A90022CE02428124C0A125B8FEF7F0097
:10175C00FEC006C00790022CE02429124C0A125B32
:10176C008FEFFDD0E02DFFD0E03400FE900212F0A0
:10177C00A3EFF0900215E02FFF900214E03E9002D0
:10178C0016F0A3EFF07FF07E011260A6900222EF1C
:10179C00F07FF17E011260A6900223EFF07FF27EC3
:1017AC00011260A6900224EFF07FF37E011260A676
:1017BC00900225EFF07FF47E011260A6900226EFD6
:1017CC00F07FF57E011260A6900227EFF07FF67E87
:1017DC00011260A6900228EFF07FF77E011260A63E
:1017EC00900229EFF0E4A3F0124BC97B017A027945
:1017FC001C125ECDEF6401707C900214E07004A3A7
:10180C00E0640E700BC2AC12191B1222C8D2AC22AF
:10181C00900214E064027004A3E0640E7057C2AF2F
:10182C00C2A0C2A1FFFE12610FE490021AF0A3F055
:10183C00900218F0A3F0125CF3900211EFF0FD90FF
:10184C00021AE0FEA3E0FF125AE490021BE004F03F
:10185C00700690021AE004F0900219E004F0700691
:10186C00900218E004F0C3900218E0940240C712F2
:10187C00191B75C720124BC97BFF7A4C794B125E32
:10188C00CDBF010612192F75C720124BC97BFF7AE9
:10189C004C7952125ECDBF010912192F12208F758F
:1018AC00C720124BC97BFF7A4C795B125ECDBF010E
:1018BC0006121943D20122124BC97BFF7A4C79696B
:1018CC00125ECDBF0106121943D20022124BC97B06
:1018DC00FF7A4C7977125ECDBF010B90022BE0FEA4
:1018EC00121964D20322124BC97BFF7A4C798312F2
:1018FC005ECD90022BE0FEBF0106121964D20422C9
:0E190C00A3E0FF900216E0FCA3E0FD1258924B
:10191A002290022BE0FEA3E0FF900216E0FCA3E077
:10192A00FD1258922290022BE0FEA3E0FF900216CD
:10193A00E0FCA3E0FD1258922290022BE0FEA3E005
:10194A00FF900216E0FCA3E0FD12589222FF9002DB
:10195A002BE03400FE125B8FEF22A3E0FF90021609
:09196A00E0FCA3E0FD12589222FA
:105CF3009002EFE0FEA3E0FF125B8F9002F0E0045E
:105D0300F070069002EFE004F09002EFE0B4780A3E
:0A5D1300A3E0B400057470124C13F5
:015D1D002263
:105BBD00AD079002EFE0FEA3E0FF125E699002F0E8
:105BCD00E004F070069002EFE004F09002EFE0B414
:0D5BDD00580AA3E0B400057450124C1322C6
:105ECD0090022D124C1B124BE06014125CF3124B1E
:105EDD00E06F60037F002290022E124BF180E77F6E
:025EED00012290
:065D730090023D124C1BE2
:105D7900E4A3F090023D124BE3FF6011125BBD906A
:105D8900023E124BF1900240E004F080E69002409E
:025D9900E0FF29
:015D9B0022E5
:1022C800C29690023B124C24125B8FEF7F00FEC037
:1022D80006C00790023CE024211224BEFDD0E02D68
:1022E800FED0E0900239124C3A90023CE0242412CD
:1022F80024BE7F00FEC006C00790023CE02425FFF4
:1023080090023BE03400FE125B8FEFFDD0E02DFF22
:10231800D0E0900237124BF8124BD8E4900231F01B
:10232800A3F07BFF7A4C798F1224CBE4900233F030
:10233800A3F090022FF0A3F0900233E0FEA3E0FF99
:102348001260A690022DEFF0125BBD900234E004FB
:10235800F07006900233E004F0900230E004F07070
:102368000690022FE004F0C390022FE0940240C8C8
:10237800900232E02400F0900231E03402F07A60FA
:1023880079161224E1EFF07A4C79961224E1E004F0
:10239800F0E004F0E51312244BE490022EF09002D2
:1023A800DFE0FEA3E0FF900235EEF0A3EFF07C0340
:1023B8007DE812037BEF1224EAF07D641224797D14
:1023C8000A122479900235E0FEA3E0FF7C007D0A22
:1023D80012037BED12244BE490022EF09002DDE014
:1023E8001224EA12249B1257D3EF64017017FF12CC
:1023F8005156BF01087B017A017903800E7BFF7A71
:102408004C799980067BFF7A4C79991224CB124734
:10241800F27B017A0279CE125D7390022EEF1224BC
:102428009B90023BE0FEA3E0FF900231E0FCA3E0BA
:10243800FD900238E02DFD900237E03CFC125A6610
:02244800D2962A
:10244A00222430FF125BBD90022EE004F07BFF7A5B
:10245A004C7996125D7390022EE004F0E004F0E0ED
:10246A00FF900232E02FF0900231E03400F0229027
:10247A000235E0FEA3E0FF7C0012037B7C007D0AAC
:10248A0012037BED2430FF125BBD90022EE004F0B4
:10249A0022F07BFF7A4C7996125D7390022EE0044B
:1024AA00F0E004F0E0FF900232E02FF0900231E019
:1024BA003400F022FF90023BE03400FE125B8FEF03
:1024CA0022125D7390022EEFF0900232E02FF0900C
:1024DA000231E03400F0227BFF125D7390022E225B
:0C24EA002430FF125BBD90022EE00422A3
:1057D3007F0012580A40037F01227401FFFE12600A
:1057E300A6EFD3940040037F01227F0212580A40A0
:1057F300037F01227F037E011260A6EFD394004052
:10580300037F01227F00227E011260A6EFD3940062
:015813002272
:1049170090020E7406F0A3E4F020133C124C33D23D
:10492700967D01FF7E06125E697DEA7F047E061290
:104937005E697D607F057E06125E697D011249937F
:10494700BF130C7D021249936414703FD213227D6A
:10495700107F017E06025E697F037E06125B8F90E1
:10496700020DEFF0601724E4600F2405701D90021C
:10497700EE7401F0C2960216DC7D0880027D107F7E
:0B498700017E06125E69124C32D296CF
:10499200227F017E06125E697F037E06125B8F9084
:0549A200020DEFF02200
:0933D90090022C124C1BA3EDF034
:1033E2009002EEE070030234EC900237124C241289
:1033F2005B8FEF7F00FEC006C007900238E02421F9
:103402001234EDFDD0E02DFED0E03400900233F016
:10341200A3CEF0900238E024241234ED7F00FEC0E7
:1034220006C007900238E02425FF900237E03400FE
:10343200FE125B8FEFFDD0E02DFFD0E09002311243
:103442004BF8900235F0A3EFF090022FE07038A312
:10345200F090022C124BE3FD6073900235E0FEA364
:10346200E0FF1234FA7006900235E004F0124BEEDF
:10347200900230E004F0900235E0B458D4A3E0B4F6
:1034820000CF124C4180CA90022FE0A3F09002308C
:10349200E06034900235E0FEA3E0FF90022C124B74
:1034A200E3FD1234FA7006900235E004F0124BEE9E
:1034B200900230E014F0900235E0B458D0A3E0B4AA
:1034C20000CB124C4180C690022FE0A3F09002374D
:1034D200E0FEA3E0FF900230E0FD900232E02DFD1D
:0A34E200900231E03400FC125A663B
:1034EC0022FF900237E03400FE125B8FEF22125E57
:0834FC0069900236E004F022A1
:09625500FF9002E4E03400FE2297
:0C621100208103024CCCE49002FEF0223D
:06627700E49002FEF0229B
:10425C009002E47407F0A3E4F02402FFE43407FEB8
:10426C00125B8F9002E1EFF07D0212000EEF640101
:10427C0060030243139002E5E0240212625590029F
:10428C00E1E04404FD125E699002E5E0242612434D
:10429C00147F00FEC006C0079002E5E024271243FD
:1042AC0014FDD0E02DFED0E034009002E2F0A3CE5D
:1042BC00F09002E5E02428126255125B8FEF7F002C
:1042CC00FEC006C0079002E5E02429126255125B7D
:1042DC008FEFFDD0E02DFFD0E03400AD07FC54078C
:1042EC00FEE42FFFEE3478FEE4B50704EEB4800054
:1042FC009002E4E0FEA3E0FF9002E3E02DFD9002CB
:07430C00E2E03CFC125892B4
:0E43130022FF9002E4E03400FE125B8FEF22E6
:104CCC007F317E001260A6EF60769002E87407F0E8
:104CDC00A3E4F09002FEE0703F7D02FF7E07125EBF
:104CEC00697DEA7F047E07125E697D6A7F057E0717
:104CFC00125E697D017F017E07125E697F037E076C
:104D0C00125B8FBF22099002FE7401F002425C7D9F
:104D1C00107F017E07025E697F027E07125B8FEFB8
:104D2C0030E31D9002E6A3E04408FD7F027E0712EB
:104D3C005E697D107F017E07125E69E49002FEF0D1
:014D4C002244
:0B621D0090020DEBF0A3EAF0A3E9F003
:016228002253
:09625E00FF90023DE03400FE2235
:10000E00AE05EFA806088002C313D8FC30E0037FCC
:05001E0001227F002219
:10350400D294C290C280126197D2807F101235EF9C
:103514007F0F7E00125E697F111235EF7F107E00EF
:10352400125E697F121235F77F117E00125E697F89
:10353400131235F77F127E00125E697F141235FF75
:103544007F057E00125E697F151235FF7F067E00BF
:10355400125E697F161236077F077E00125E697F4E
:10356400171236077F087E00125E697F1812360F25
:103574007F017E00125E697F1912360F7F027E0082
:10358400125E697F1A1236177F037E00125E697F0E
:103594001B1236177F047E00125E697F1C12361FD1
:1035A4007F097E00125E697F1D12361F7F0A7E002E
:1035B400125E697F1E1236277F0B7E00125E697FC2
:1035C4001F1236277F0C7E00125E697F207E001258
:1035D40060A6AD077F0D7E00125E697F217E00121A
:1035E40060A6AD077F0E7E00025E697E001260A6B3
:1035F400AD07227E001260A6AD07227E001260A6EF
:10360400AD07227E001260A6AD07227E001260A6DE
:10361400AD07227E001260A6AD07227E001260A6CE
:0B362400AD07227E001260A6AD072259
:0E619700E4F5D875F9FDF5E9D2DE30DFFD2222
:105FE200E4FEEF30E704D2918002C291D290EF2515
:095FF200E0FFC2900EEEB408E9D4
:015FFB002283
:075E6200FFE43EFEA3E0FD9A
:105E6900AB07AA06C2947FF0125FE2EAFF125FE273
:0D5E7900AF03125FE2AF05125FE2D2942288
:045B8F00AD07AC06AC
:105B9300C2947F0F125FE2ECFF125FE2AF05125F68
:105BA300E2E4FFFED290EF25E0FF3093034401FFD0
:095BB300C2900EEEB408EDD2948C
:015BBC0022C6
:105A660090023FECF0A3EDF090023DEEF0A3EFF0D4
:105A76002424125E6290023EE0242512625E9002A9
:105A860040E0FD125E6990023EE0240112625E7DF6
:045A960020025E6923
:1058920090022FECF0A3EDF090022DEEF0A3EFF0CA
:1058A2002428125E6290022EE02429FF90022DE04D
:1058B2003400FE900230E0FD125E6990022EE02478
:0E58C20001FF90022DE03400FE7D40025E6981
:10566400E0FAA3E0FBFFAE0212037BEF2430FF90CD
:10567400020DE024B0F582E43402F583EFF09002E9
:105684000DE004F0227C00AF03AE0212037B7C0029
:105694007D0A12037BED22E024B0F582E43402F5A6
:0D56A4008322E0FAA3E0FB7C007D0AFF22D8
:102FE100125D49EF7002FF227FCC125FAB7F44126A
:102FF1005FAB30C6FD125D49EF7002FF227FCC123C
:103001005FAB7FBE125FAB125EEF9002B8E4F0A33C
:10301100EFF0125EEF9002B6E4F0A3EFF0E490025D
:103021000DF090020DE0FFC39406500C74B02F1206
:10303100569EE412568180EA9002B6A3E0FF30E783
:103041001DD214FE9002B9E02400FF9002B8E03EC8
:10305100FEEFF4FFEEF4FEEF2401FDE48012C21452
:103061009002B7E0FE9002B9E02400FD9002B8E0C2
:103071003EFCE4120151E4FBFA7920783F1200464C
:1030810012018A90020EEEF0A3EFF0E490020DF02F
:1030910030140812569B742D125681C390020FE012
:1030A100946490020EE09400500C1256A6AE0212E7
:1030B100037BEF02311AC390020FE094E890020EF5
:1030C100E09403502C7C007D641256647D0A1256F4
:1030D100892430FF12567612569B742E125681A304
:1030E100E0FEA3E0FF1256922430FF90020D023160
:1030F10034C390020FE0941090020EE094275041E7
:103101007C037DE81256647D641256892430FF12D7
:103111005676A31256A612568D12567012569B74ED
:103121002E1256817C007D0AAF03AE0212037BEDA5
:103131002430FF12567612569B74431256817F013A
:03314100227F00EA
:013144002268
:0761350012613CD2C67F019C
:0B613C00AE071FEE6004000080F6229A
:105D4900D2D7C2C67FF012613C7FF012613CD2C645
:105D59007F3C12613CA2C67FF012613C7FB41261A4
:0A5D69003C20D7037F01227F0022B7
:105EEF00E4FDFCEDC313FDC2C67F0112613530C660
:105EFF0004ED4480FD7F3C12613C0CECB408E4AF30
:015F0F00058C
:015F1000226E
:025FAB00AD0740
:105FAD00E4FCC2C67F0112613CEDC313FD92C67FB6
:095FBD003C1261350CECB408E95A
:015FC60022B8
:0D61EA000D0A495320202D3E52463A200058
:1058D000F00C74002CF582E43400F58374A0F00C15
:1058E00074002CF582E43400F5832274802DF58257
:1058F000E43400F583E02274812EF582E43400F56F
:0E59000083E022EEF00C90021EE004F00D2277
:10551600E4FF74802F1258EE643E600A0FEFD394B6
:105526000C40EF7F6322E4FE74802E1258EEFD6479
:105536003E6030ED642D7028C3EF9EB40208125809
:10554600F7C39430FF221258F724D075F00AA4FF4F
:1055560074822EF582E43400F583E024D02FFF22F6
:055566000E80C57F006E
:01556B00221D
:0D61DD007F2E7E001260A69002FFEFF022E0
:1032A6009002FFE070030233D8125516EF64637084
:1032B600030233D8E4FE74802E1258EE643E600892
:1032C6000EEED3940C40EF227D069000007440F081
:1032D600A3DDFC7D060EE4FC74802E1258EEFB6422
:1032E6002C6012EB25E0FB1258E0EBF00C0EEED34F
:1032F600941240E4229000067460F00C7D06900063
:10330600077440F0A3DDFC7C07EFD39400401AE479
:10331600FD90021EF01258EBFE642D6026EE25E0AD
:10332600FE1258E012590380ECE4FD90021EF012E2
:1033360058EBFE643E600CEE25E0FE1258E0125992
:103346000380ECEF25E0446090000DF07C0E1258EF
:10335600E074A81258DE74861258D074921258D0AF
:1033660074401258DE74E11258DE74031258DE748B
:10337600F0F00CE4FD1258EB643A60080DEDD394BE
:103386003240F2220D1258EBFF60091258E0EFF0BE
:103396000C0D80F1AF04900100EFF0FD7B017A0087
:1033A60079001250807B017A007900900100E0FDDF
:1033B600123A477B017A007980122CAC7BFF7A6146
:1033C60079EAE4FD1233D97B017A007980E4FD12B3
:0233D60033D9E9
:0133D80022D2
:104F3600E0FF90021FE0FBA3E0FAA3E0F990022352
:104F4600E0F58275830022EF120347900223E00406
:104F5600F02274002FF582E43400F583E0C3139049
:104F66000225F0642022EF4430FFF090021FE0FBA0
:104F7600A3E0FAA3E0F922E0541EC313900226F040
:104F8600D3940022900226E024F6F0E04430222456
:104F960006F582E43400F58322900222E004F02232
:0B2CAC0090021FEBF0A3EAF0A3E9F098
:102CB700E4900223F09002227407F0900222E0FFD2
:102CC700C3940D5010124F586006124F36124F4DD5
:102CD700124F9F80E690000D124F7D402A124F3809
:102CE700742D124F4E900226E0FFC3940A5005122E
:102CF7004F6C800D124F387431124F4E124F8AFFAE
:102D0700F0124F43124F4D124F38743E124F4EE49C
:102D1700900222F0900222E0FFC394065010124F57
:102D2700586006124F36124F4D124F9F80E69000A3
:102D370006124F7D402A124F38742D124F4E9002C3
:102D470026E0FFC3940A5005124F6C800D124F38CE
:102D57007431124F4E124F8AFFF0124F43124F4DEC
:102D67009002247407F090000DE030E003022E1269
:102D7700124F38742C124F4EA3E02407F0E0900254
:102D870022F0900224E02406FFE433FE900222E0C2
:102D9700FDC39FEE6480F8748098501374002D1261
:102DA7004F5B6006124F36124F4D124F9F80D390E4
:102DB7000224E0FF124F95124F7D402F124F3874B7
:102DC7002D124F4E900226E0FEC3940A5009EE449E
:102DD70030FE124F70800D124F387431124F4E1261
:102DE7004F8AFEF0124F43EE124F4E74062F124FCA
:102DF70097E030E708124F38742A124F4E9002249A
:102E0700E0124F95E020E003022D77124F38743A15
:102E1700124F4EA3E02409F0E0900222F090010047
:102E2700E0FF900222E0FEC39F501574002EF5824A
:102E3700E43400F583124F36124F4D124F9F80DD59
:102E4700124F38740D124F4E124F46740A124F4EDE
:072E5700124F46E40203479D
:105C44000D0A4E4D45412034383030204F55543ADA
:105C540020000D0A4E4D45412039363030204F5535
:0C5C6400543A200024475057504C2C00AC
:1059C000F583E0FF900211E02480F582E43400F5D5
:1059D0008322742CF0900211E004F022900211E076
:1059E000FF900210E0FEC322900210E004F022F5C6
:0859F00082E43400F583E0229B
:0519730090020FEFF0EF
:10197800900212740DF0E4A3F0900213E0C39403F4
:101988004003021BEE900212E024001259EF20E0FF
:1019980003021BE1E4900211F0900210F090021093
:1019A800E0FFC394075011EF905C68931259C3EF9E
:1019B8001259D41259E880E5900212E024049002EA
:1019C80010F0900212E0240BFFE433FE900210E0C6
:1019D800FDC39FEE6480F8748098501474002DF550
:1019E80082E434001259C0EF1259D41259E880D257
:1019F8001259C41259D2A3E0FF240BF582E4340033
:101A0800F583E0FE1259C4EE1259D41259C712597F
:101A1800D2EF240D900210F0900212E0FF2415FD81
:101A2800E433FC1259E19DEC6480F87480985013FB
:101A380074002E1259EFFE1259C4EE1259D41259DD
:101A4800E880D51259C41259D274152FF582E4349E
:101A5800001259C0EF1259D41259C71259D2900224
:101A6800107407F0900210E0FFC3940D5019740031
:101A78002F1259EFC313FF642060071259C4EF12E5
:101A880059D41259E880DD90000DE0541EC313FFAD
:101A9800D3940040301259C4742D1259D4EFC39412
:101AA8000AEF5002801575F00A842430FE1259C4DA
:101AB800EE1259D4EF75F00A84E5F02430FF12597C
:101AC800C7EF1259D41259C4742A1259D4E4FF909A
:101AD800021004F0900211E0FE14FD900210E0FCE8
:101AE800C39D500E74802C1259CAE06FFF1259E83A
:101AF80080E2EFC4540FFDC3940AED500C2430FD6E
:101B080074802E1259CAED80072437FE1259C4EE8C
:101B18001259D4EF540FFFC3940AEF5004243080B5
:101B28000224371259C3EF1259D41259C4740D1232
:101B380059D41259C7740A1259D41259C7E4F090EB
:101B4800020FE014602E14604924026003021BEEA9
:101B5800E4900210F01259DC9F501074802E125934
:101B6800CAE0FF1260781259E880EA7BFF7A5C7954
:101B780044021BD1E4900210F01259DC9F500B7400
:101B8800802E1259CA121BEF80EF7BFF7A5C7956C0
:101B98008037E4900210F01259DC9F501074802EA8
:101BA8001259CAE0FF12624B1259E880EAE4900227
:101BB80010F01259DC9F500B74802E1259CA121B58
:101BC800EF80EF7BFF7A5C7956E4FD1233D97B0115
:101BD8007A007980E4FD0233D9900212E02407F0FC
:061BE8001259E802198108
:0D1BEE0022E0FF12608F900210E004F02250
:106061000D0A524620494E203A20000D0A4953207C
:076071004F5554203A2000B6
:105FFC00900100E0FF90020EE0FEC39F2274002E81
:0A600C00F582E43400F583E0FF2282
:10455D00C2A07F847E011260A6BF01077F021219DF
:10456D0073804E7FC012624BE4FF12624BE49002E7
:10457D000EF0125FFC500E12600912624B90020E8B
:10458D00E004F080ED7FC012624B7FC012608FE4BB
:10459D00FF12608FE490020EF0125FFC500E12605D
:1045AD000912608F90020EE004F080ED7FC0126062
:1045BD008F7B017A007980122CAC7A60796112457B
:1045CD00FDE4FD1233D97F357E001260A6BF0115C3
:1045DD007B017A00798012374A7A60796C1245FD39
:1045ED00E4FD1233D9121BFBD2A0125BEA024AC0C2
:0E45FD007BFFE4FD1233D97B017A0079802226
:1053A400F8900245E0FCA3E0FDA3E0FEA3E0FF12B9
:1053B4000471E47B0AFAF9F8120471EB2430FF90CB
:1053C400024DE024CEF582E43402F583EFF090023E
:1053D4004DE004F0E024CEF582E43402F583227B30
:1053E400E87A03F9F8900245E0FCA3E0FDA3E0FEAF
:0E53F400A3E0FF020471F090024DE004F022ED
:0D61F700759180759280759D8075BCA02209
:105A2F00E4F5BDF5BEE5BC54E044084FF5BC0000FD
:105A3F0000007DFAE5BC30E41753BCEFAFBDEF7546
:105A4F00F004A4FFACBEEC7A002FFFEA35F0FE2283
:065A5F00DDE27E037FFF83
:015A6500221E
:1047F2007F07125A2FE4FCFD900249120522E47F42
:10480200E87E80FDFC900249E0F8A3E0F9A3E0FA1B
:10481200A3E0FB1203E6E4FB7A24F9F8120471EF39
:104822002423FFE43EFEE43DFDE43CFC90024512FD
:104832000522E41253E3E4FBFAF9F8C312051170FE
:104842000890024DF07B64801BE490024DF01253FD
:10485200E3EF2430FF90024D1253D8EF1253FAE4E3
:104862007B64FAF91253A4742E1253FAE47B0AFA07
:10487200F91253A474561253FA90024D1253D8E40B
:034882001253FAD4
:014885002210
:105A9A00C313F04480F0A3E004F0E022E4F5D875E3
:105AAA00F9FD75E908D2DE227B017A0079009001BE
:105ABA0000E0229002EAE0640322F583E0FF90020C
:045ACA00FAE06F226D
:105C7000308303D2C022C2C07F827E011260A69010
:105C800002EBEFF0C2AC1246B490020DEFF01260DE
:0B5C9000D390020DE0B4010312455D4B
:015C9B0022E6
:1046B400124EC1125ABD60037F00229002ECE064E6
:1046C4007E60037F00221250EC9002ECE0FEB47E88
:1046D40008125ABD60F07F0022E4900100F0E0244B
:1046E40000F582E43400F583EEF0900100E004F07C
:1046F400E490020EF01250EC125ABD60037F0022C7
:10470400900100E0FED3947840037F00229002ECF5
:10471400E0FF74002EF582E43400F583EFF090019D
:1047240000E004F0EFB47ECD90020EE004F09002BD
:10473400EBE0FF90020EE0D39F40BA900100E0C38B
:104744009F14F012590EBF01037F0122125B31BF87
:0747540001037F01227F0039
:01475B00223B
:10590E00125AB224FEFD125080900100E0FE24FED9
:10591E00F582E434FF125AC460037F002274FF2E16
:10592E00F582E434FFF583E0FF9002F9E06F600347
:0D593E007F0022900100E024FEF07F012296
:105B3100125AB214FD125080900100E024FFF58248
:105B4100E434FF125AC460037F00229002F9E0643A
:0F5B51007E60037F0022900100E014F07F0122AC
:104EC100E49002EAF09002ECF0A284920DA3F0903B
:104ED100020FF012616A9002ECE0FFC313F0A3E04D
:104EE100B4061690020FE004F0E0B4030C9002EA5D
:104EF1007403F0E49002EDF022E49002EDF0C20EB2
:104F0100200ED012627D20DF183083079002EA74F0
:104F110004F022A284300D01B350EBA284920DD291
:104F21000E200EDC9002ECE0125A9AB407D29002E5
:044F3100EA7405F029
:014F35002259
:1050EC00E490020FF090020FE0C39408505B126240
:1050FC007D20DF1E3083079002EA7404F022A28424
:10510C00300D01B35008A284920DD20E8004C20E51
:10511C0080DF200E149002ECE0FF125A9AB40707BD
:10512C009002EA7405F022801812616A9002EDE098
:10513C00B40504E4F080AE9002ECE0C313F0E4A3F9
:09514C00F090020FE004F0809CD9
:015155002237
:0E3A470090021FEBF0A3EAF0A3E9F0A3EDF06C
:103A5500C2AC7F807E011260A6900225EFF0C2867F
:103A6500D287D282D285E49002EDF0900223F090C5
:103A75000225E02401FFE433FE900223E0C39FEE1C
:103A85006480F87480985014E4A3F0123B31E0C3CD
:103A9500942640F7900223E004F080D3E4900224BA
:103AA500F0900222E0FF900224E0C39F5024900290
:103AB5001FE0FBA3E0FAA3E0F9120301FF12528411
:103AC500900220E475F0011203D0900224E004F086
:103AD50080CF9002FAE0FF1252849002F9E0FF12C3
:103AE5005284E4900224F0123B31E0C3940540F780
:103AF500D286C287C2821260D37F817E011260A600
:103B0500900226EFF0D394004021E4900224F09037
:103B15000226E0FF900224E0C39F500F7F057E0040
:0B3B2500125F8D900224E004F080E4A9
:0D3B3000227F7E125284900224E004F022D5
:05528400900227EFF08D
:10528900BF7E04D20C8002C20CE4900228F0900286
:1052990027E054017004B28580269002EDE004F005
:1052A900200C047F0180027F009002EDE0B4050428
:1052B9007E0180027E00EE5F600A120003B285E47F
:1052C9009002EDF0900227E0FFC313F01200039063
:0B52D9000228E004F0E0C3940840B39A
:0152E40022A7
:07000300125AA630DFFD22B6
:04627D00125AA622E9
:0F616A00E4F5D875F9FE75E980D2DE30DFFD224D
:07627000C282D286C2872220
:105BEA007F8F7E011260A6EF60227F1C7E02EF1F6C
:105BFA00AC0670011E4C6012B2C3E4F5D875F9FF09
:0C5C0A0075E956D2DE20DFE680FBD2C335
:015C1600226B
:1024F600000011892312329B462457AD653674BFFE
:102506008C489DC1AF5ABED3CA6CDBE5E97EF8F7AD
:10251600108101083393221A56A5472C75B7643EDD
:102526009CC98D40BFDBAE52DAEDCB64F9FFE8768D
:102536002102308B02101399672676AF443455BDBD
:10254600AD4ABCC38E589FD1EB6EFAE7C87CD9F56D
:102556003183200A1291031877A7662E54B5453C9D
:10256600BDCBAC429ED98F50FBEFEA66D8FDC9744D
:102576004204538D6116709F042015A9273236BB7D
:10258600CE4CDFC5ED5EFCD7886899E1AB7ABAF32D
:102596005285430C7197601E14A1052837B3263A5D
:1025A600DECDCF44FDDFEC5698E98960BBFBAA720D
:1025B6006306728F4014519D252234AB063017B93D
:1025C600EF4EFEC7CC5CDDD5A96AB8E38A789BF1ED
:1025D6007387620E5095411C35A3242A16B107381D
:1025E600FFCFEE46DCDDCD54B9EBA8629AF98B70CD
:1025F60084089581A71AB693C22CD3A5E13EF0B7FD
:10260600084019C92B523ADB4E645FED6D767CFFAC
:1026160094898500B79BA612D2ADC324F1BFE036DC
:1026260018C109483BD32A5A5EE54F6C7DF76C7E8C
:10263600A50AB48386189791E32EF2A7C03CD1B5BC
:10264600294238CB0A501BD96F667EEF4C745DFD6C
:10265600B58BA40296998710F3AFE226D0BDC1349C
:1026660039C3284A1AD10B587FE76E6E5CF54D7C4C
:10267600C60CD785E51EF497802891A1A33AB2B37C
:102686004A445BCD695678DF0C601DE92F723EFB2C
:10269600D68DC704F59FE41690A98120B3BBA2325C
:1026A6005AC54B4C79D7685E1CE10D683FF32E7A0C
:1026B600E70EF687C41CD595A12AB0A3823893B13C
:1026C6006B467ACF485459DD2D623CEB0E701FF9EC
:1026D600F78FE606D49DC514B1ABA02292B983301C
:1026E6007BC76A4E58D5495C3DE32C6A1EF10F78CC
:0550800090021FEDF09D
:1050850074FFA3F0A3F090021FE0D39400403F12F9
:105095000301FF900220A3E06F25E0FFE433FE74D7
:1050A500F62FF58274243EF583E493FC740193FD99
:1050B500900220E0FFECFEED6FFFEEF0A3EFF09025
:1050C500021FE014F0740129F9E43AFA80B890025D
:1050D50020E0FEA3E0F4FFEEF4FCEF9002FAF0AE60
:0650E50004EE9002F9F058
:0150EB0022A2
:105F8D00EF4E6019EF1FAC0670011E4C600FE4F56B
:0E5F9D00D875F94CF5E9D2DE20DFE980FB2251
:0E61A5000D0A444947492D3E5246203A20003B
:10534500EE2402FFE433FE7C007D07120369AC0600
:10535500AD0722900216E02417F582E43402F583A6
:105365002274062DF58274003CF583222400F58213
:10537500E43400F583227B017A007900900100E096
:10538500FD2290020FE0FFA3E0FEC39F22F09002F2
:0F53950013E004F0222418F582E43402F5832299
:104AC0007F0DE490020FF074002F125373E020E08A
:104AD0001174072FFF90020FE004F0E0D39406401A
:104AE000E62290020FE0605DE4900211F090021067
:104AF000F0125387501B1253457FB07E011241952F
:104B0000BF02069002117401F0900210E004F080E0
:104B1000E0E4900210F0125387501B1253457FB708
:104B20007E01124195BF02069002117401F09002BD
:104B300010E004F080E0900211E0B401087F0E1252
:054B40003D2812522285
:014B4500224D
:0E419500900212EEF0A3EFF0A3ECF0A3EDF019
:1041A300E4A3F0900216E0FFC39406502C90021390
:1041B300E02FFF900212E03400FE1260A6EF7008B9
:1041C3001253587440F08009EF25E0FF125358EF63
:1041D300F0900216E004F080CAE4900216F0900218
:1041E30016E0FFFD900215E02DFD900214E034006F
:1041F300FC74002DF58274003CF583E0FE74172FE8
:1042030012535EE06E60037F0022900216E004F01A
:10421300E0B406CA900214E0FCA3E0FD24061253A6
:1042230069E0FE541EC313FF70037F01221FEF25B5
:10423300E0FF125366EE54E1F0125366E04FF0EFE5
:104243007014900214E0FEA3E02406F58274003E8D
:08425300F583E04480F07F02D6
:01425B002240
:053D2800900212EFF013
:103D2D00900100E0D394784003023E16E490021611
:103D3D00F0A3F0FFFE1260A6EF7003023E16E490B2
:103D4D000216F0A3F0900213F0900216E0FEA3E02D
:103D5D00FF1260A6EF25E0900215F070037440F09D
:103D6D00900215E0FF900213E012539AEFF09002CB
:103D7D0017E004F07006900216E004F0125393E081
:103D8D00C3940640C47F877E001260A6EF25E044F1
:103D9D00E090021EF0900214E004F0900100E0FFAC
:103DAD00900215F0900212E014FEC3EF9E900214E3
:103DBD00F0E4900213F0900214E0FF900213E0C3C0
:103DCD009F5020900215E0FF125371E0FE74072FF3
:103DDD00F582E43400F583EEF0900215E0141253F1
:103DED009280D3E4900213F0900213E0FF12539AE5
:103DFD00E0FE900212E02F125371EE125392E0B4D6
:093E0D0007E6900100E02407F033
:013E16002289
:105222007F887E011260A6900213EFF0D3940040B3
:1052320021E4900212F0900213E0FF900212E0C308
:105242009F500F7F057E00125F8D900212E004F0E6
:1052520080E4C2A112537B12508012537B123A4750
:105262007B017A007980122CAC7BFF7A6179A5E40C
:10527200FD1233D97B017A007980E4FD1233D9D251
:01528200A18A
:015283002208
:0F617900E4F5D875F9FF75E940D2DE30DFFD227D
:0F618800E4F5D875F9FF75E9A0D2DE30DFFD220E
:10607800C2C41261797E08EFC313FF92C41261791A
:07608800DEF5D2C4026179CC
:10608F00C2C41261887E08EFC313FF92C4126188E5
:07609F00DEF5D2C4026188A6
:0962670090020DE0FF14F0EF229B
:10556C0090020DEDF025E0F0EF24FE60160470269D
:10557C00126267600BB2B77F017E00125F8D80F004
:10558C00D2B722126267600BB2967F017E00125F67
:10559C008D80F0D296221262676011B2B7B296B2C9
:1055AC00A0B2A17F017E00125F8D80EAD296D2B7A5
:0555BC00D2A1D2A022E3
:106016002047572D313030302046573A20312E3028
:0A602600382000563A312E303800C1
:105C9C009002BEE508F0A3E509F0229002C0E50AE7
:105CAC00F0A3E50BF0229002BCE50CF0A3E50DF09F
:0C5CBC00229002BAE50EF0A3E50FF022E2
:1060BD00125460C2B6125CC8126241125C7012506A
:0660CD001312603080EFA9
:105E150020A2237F017E00125F8D20A21912208F00
:105E2500C2AFC2A0C2A130A2FD7F017E00125F8D6C
:075E350030A2F375C7202223
:103B3D00125B60EF7010C2AFC2A0C2A112208FD273
:103B4D00A1D2A075C7207F80123C257F00FEC00644
:103B5D00C0077F817E001260A6EFFDD0E02DF50934
:103B6D00D0E03400F5087F827E001260A6EF7F0062
:103B7D00FEC006C0077F83123C25FDD0E02DF50B5E
:103B8D00D0E03400F50A7F00123C1BC006C007745C
:103B9D00010FFE1260A6EFFDD0E02DF50DD0E03443
:103BAD0000F50C7F02123C1BC006C0077F03123CC0
:103BBD002CFDD0E02DF50FD0E03400F50E7F8312F3
:103BCD003C2C7004D2A78002C2A77F907E011260A8
:103BDD00A6EF7F00FEC006C0077F917E011260A692
:103BED00EFFDD0E02DF511D0E03400F510125C9C06
:103BFD00C200125CA7C201125CB2C204125CBDC24B
:103C0D00039002C2E510F0A3E511F0C202227E017D
:103C1D001260A6EF7F00FE227E001260A6EF227ECC
:063C2D00011260A6EF2267
:1054600043B70243B80243B710125E15126270755B
:10547000BBFFC2C4125F6F126281126277D2B7D2D1
:10548000961261F7123B3D1261C11262041261DD96
:10549000123950122FE1122FE17D027F0312556C59
:1054A000125BEAC28C9001017414F0C28CC28D753B
:0C54B0008C4CE4F58AD28CD2A9D2AF2239
:03000B00023FE7CA
:103FE700C0E0C0F0C083C082C0D075D000C000C0A0
:103FF70001C002C003C004C005C006C007C28CC20E
:104007008D758C4C758A00D28C900101E014F0E01C
:1040170060030240A57414F0E5094508601A900290
:10402700BFE024FFF09002BEE034FFF0E07002A38F
:10403700E07005125C9CD200E50B450A601A9002FD
:10404700C1E024FFF09002C0E034FFF0E07002A36B
:10405700E07005125CA7D201E50D450C601A9002CD
:10406700BDE024FFF09002BCE034FFF0E07002A353
:10407700E07005125CB2D204E50F450E601A90029B
:10408700BBE024FFF09002BAE034FFF0E07002A337
:10409700E07005125CBDD203126159125F51D0075F
:1040A700D006D005D004D003D002D001D000D0D0A4
:0940B700D082D083D0F0D0E032B9
:1049A700C0A80178FFFFFF00C0A801010008DC01D3
:1049B7000203CDE9232E810F292392E5A2B6746560
:1049C7007374000000303030000000333131312E75
:1049D70038314E000031323133312E323245004703
:1049E700572D3130303020424541434F4E20000093
:1049F700000000000000000000000000003331311B
:104A0700312E37304E000031323133312E303045C0
:104A17000047572D31303030205758200000000014
:0F4A270000000000000000000000000000000080
:1058530090022DE0FEA3E0FFE4FD125AE4E004F021
:105863002290022DE004F02290022DE0FEA3E0FF3F
:105873002275C65A75C6A522ECF5C3AF058FC4229F
:0F58830090022D7401F0A32290022DE4F0A322D5
:105B60007F1C125B8860037F00227F1D125B8864AC
:105B70000860037F00227F1E7E001260A6EF64DCB7
:0F5B800060037F00227F01227E001260A6EF22C9
:0E61B300E4F5C7F5C5F5C675C3FF75C4FF2238
:0460A600AD07AC0690
:1060AA0075C78275C50112587B12587400AFC212A7
:0260BA0061B3D0
:0160BC0022C1
:10610F00AD07AC0612587B75C78275C5031258745C
:03611F000261B367
:105C1700AD07AC0675C78275C50212587B12030122
:105C2700F5C2125874000DBD00010C740129F9E486
:0D5C37003AFA900234E014F070E00261B31C
:105ACE007F81125AE47F82125AE47F83125AE47F56
:065ADE0084125AE47F85EA
:105AE400AB07AA0675C78275C502EAF5C3AF038F73
:0C5AF400C4AF058FC2125874000261B3E9
:10208F00E4FFFE12610F7BFF7A4979C59002347429
:10209F0007F0E4FF125C177D0A7F07125AE47BFFFB
:1020AF007A4979CC9002347407F07F09125C177A61
:1020BF004979A79002347412F07F10125C177A4995
:1020CF0079B9900234740CF07F22125C17E4FD7F13
:1020DF002E125AE47F2F125AE47F30125AE47F31C6
:1020EF00125AE47F32125AE47F33125AE47F3412C9
:1020FF005AE47F35125AE47F40125AE47F80125A15
:10210F00E4125ACE7D0A7F87125AE47D217F88120E
:10211F005AE47D2F7F89125AE47D237F8A125AE475
:10212F0012588B7490F0E4FCEC9049D293FD600E42
:10213F0012586B12585D70031258640C80EA1258D3
:10214F0053700312586412588B74A0F0E4FCEC9097
:10215F0049DC93FD600E12586B12585D70031258D4
:10216F00640C80EA125853700312586412588B741F
:10217F00B0F0E4FCEC9049E693FD600E12586B1240
:10218F00585D70031258640C80EA12585370031292
:10219F005864E4FDFF7E01125AE4E404FF125AE48E
:1021AF007F02125AE47F03125AE47F04125AE47F2B
:1021BF0005125AE47F06125AE47D0D7F07125AE486
:1021CF00E4FD7F0B125AE47D3D7F08125AE47D2F08
:1021DF007F09125AE47D5F7F0A125AE41258837402
:1021EF0010F0E4FCEC904A0493FD600E12586B1251
:1021FF00585D70031258640C80EA12585370031222
:10220F0058641258837420F0E4FCEC904A0E93FD4E
:10221F00600E12586B12585D70031258640C80EAEE
:10222F0012585370031258641258837430F0E4FC40
:10223F00EC904A1893FD600E12586B12585D7003A4
:10224F001258640C80EA12585370031258647D01BF
:10225F007F807E01125AE41D125ACE7F86125AE4F5
:10226F007F87125AE40D7F88125AE41D7F89125A14
:10227F00E47F8A125AE47F8B125AE47F8C125AE45D
:10228F007F8D125AE47F8E125AE40D7F8F125AE41B
:10229F00E4FCEC2490FFE43401FEE4FD125AE40C5C
:1022AF00ECB430EEE4FCEC24F0FFE43401FE7D30BE
:0822BF00125AE40CECB408EE25
:0122C70022F4
:0E61CF000D0A42542D3E52462F49533A2000ED
:106122007B017A007900900100E0FD227B017A0078
:036132007980224F
:0E61C100759850758921758DFDD28E0260D3C0
:1060D300C2ACC20FE4900206F07F80900186E4F028
:0560E300A3DFFCD2ACBC
:0160E8002295
:03002300024FA6E3
:104FA600C0E0C083C082C0D0309906C299D21080BA
:104FB60053309850C298300F07900206E4F08044B0
:104FC600900206E02486F582E43401F583E599F043
:104FD600900206E004F0E599B4C01CE0D3940E40BC
:104FE60016900186E0B4C008A3E07004D20F8014C6
:104FF600C20F900206E4F0900206E0D3947E4004CD
:0D500600C20FE4F0D0D0D082D083D0E032D1
:10501300300F69C2A1E4900100F07F02900206E024
:1050230014FEEFC39E502174862FF582E43401F5FC
:1050330083E0FE74FE2FF582E434FFF583EEF090F7
:105043000100E004F00F80D412612212508012613B
:1050530022123A4712612E122CAC12612E12374AD9
:105063007BFF7A6179CFE4FD1233D912612EE4FD1F
:0C5073001233D9D2A1E4900206F0C20F63
:01507F00220E
:0A624B00C2108F993010FDC210221E
:104D4D000D0A4750532D3E4750524D43203A2020D7
:104D5D00494F312020475053204E4F20636F6E6EC8
:104D6D00656374210D0A000D0A4750532D3E4750BF
:104D7D00524D43203A20000D0A4750532D3E4750C7
:104D8D00524D43203A2020475053204E4F204C4F38
:104D9D00434B210D0A004750532D3E4750524D4372
:104DAD00203A20004750532D3E4750474741203A67
:104DBD002000244750524D4300244750474741009F
:1028F500E0FAA3E0FB7C037DE8FFAE0212037BEF69
:102905002430FF9002A3E02481F582E43402F583AC
:10291500EFF09002A3E004F07C007D64AF03AE020B
:1029250012037B7C007D0A12037BED2430FFE0243B
:1029350081F582E43402F583EFF09002A3E004F020
:10294500E02481F582E43402F583220F9002F4E05D
:10295500FBA3E0FAA3E0F98F8275830002031AEF67
:102965002BFBEE3AFA7D0A7C00E024D0FFE434FF2D
:10297500FE020369EFF09002A3E004F0229002D674
:10298500E0FBA3E0FAA3E0F922EF2BFFEE3AFEA36A
:10299500E090029924D0FDEC34FFCD2FFFED3EF001
:1029A500A3EFF022AA06AB077C037DE8E024D0FF65
:1029B500E434FFFE020369A3F07B017A0179032267
:1029C5009002C8E0900262F09002C9E0900263F0C4
:1029D5009002CAE0900264F09002CBE0900265F0AC
:1029E5009002CC229002C9E0900262F09002CAE007
:1029F500900263F09002CBE0900264F09002CCE08C
:102A0500900265F09002CD22E0FAA3E0FB7C007D08
:102A15000AFFAE0212037B7C007D0A12037BED24C4
:102A250030FF229002C8E0900263F09002C9E09066
:102A35000264F09002CAE0900265F09002CB22EBAE
:102A4500F0A3EAF0A3E9F022E024D075F00AA4FF90
:102A5500229002C7E024C8F582E43402F583EEF043
:102A65009002C7E004F00F229002C8E0900264F0E3
:102A75009002C9E0900265F09002CA22EF75F00A53
:102A850084E5F024302274D92DF582E43402F583EF
:102A9500EFF00C0D2290029BE0FEA3E0FF229002D6
:102AA5009DE0FEA3E0FF2224D075F064A42FFFE093
:102AB50024D02F22E0FF75F00A842430FE9002A373
:102AC500229002C8E0900265F09002C922E0FCA3C2
:102AD500E0FDC39FEC9E22ED9FFFEC9EF0A3EFF07F
:012AE50022CE
:0556B100900300EFF082
:1056B600E4F5AF9001847403F07F8C7E011260A63E
:1056C600EF7005759CFA8003759CFD43A21090034C
:1056D60000E024FF9208C207E4900185F0FF7403FE
:1056E6002FF582E43401F583E4F00F0FEFC39480C5
:0556F60040EC75AF015E
:0156FB00228C
:105D1E007F927E011260A6900296EFF024FE600E36
:105D2E0014600E24027013300210C2028009024663
:0B5D3E000B125EAABF0103124A3622BE
:105EAA003087037F00227F017E00125F8D308703D7
:105EBA007F00223087FD7F017E00125F8D3087F3DD
:035ECA007F012233
:1052E500E4FF1256B1E4900301F020071E7F017E12
:1052F50000125F8D900301E004F0E0D3942840EAAA
:10530500E4F5AF7BFF7A4D794D802EE4F5AF7BFF59
:105315007A4D7974FD1233D91229BEE4FD1233D9C1
:105325001229BE125D9CBF01091229BE123C337FB2
:1053350001227BFF7A4D7984E4FD1233D97F002267
:104A3600E4FF1256B1E4900302F0200707124AAED3
:104A460040F880407BFF7A4D79A3E4FD1233D912FA
:104A560029BEE4FD1233D91229BE125D9CBF011096
:104A66001229BE123C331229BE123858D2058002D2
:104A7600C2057F011256B1E4900302F02007091225
:104A86004AAE40F8E4F5AF227BFF7A4D79B1E4FDFA
:104A96001233D91229BEE4FD1233D91229BE123EB1
:074AA60017300503123F0267
:104AAD00227F017E00125F8D900302E004F0E0D3BF
:034ABD0094282218
:10460B0090027DE01460161460552402600302468C
:10461B00AEE4F5AF90027D04F0E4FF803F2007038A
:10462B000246B37BFF7A4D79A3E4FD1233D91229ED
:10463B00BEE4FD1233D91229BE125D9CBF011012CC
:10464B0029BE123C331229BE123858D2058002C241
:10465B0005E4F5AF90027D7402F07F010256B13094
:10466B0007467BFF7A4D79B1E4FD1233D91229BE8F
:10467B00E4FD1233D91229BE123E173006109002F8
:10468B0080E004F0E0D394054019C2068015300594
:10469B00121243E4BF010A123F02D206E4900280D9
:0946AB00F08000E490027DF02291
:10561500900103E064246007E4900185F0FF2220F7
:10562500081D90020A74FFF0A3744DF074BF12298F
:10563500BC125986BF0105D207E4F5AF7F00229061
:10564500020A74FFF0A3744DF074C61229BC1259F6
:0F56550086BF0108D207E4F5AF7F01227F002254
:105E8600E4900294F0A3F0900269F0900267F0901B
:105E9600027FF090027EF0C205900280F0C206906A
:045EA600027DF02267
:063E17009002C4122A44CF
:103E1D00E4FFFE9002C4122954FD6009B42C010E7A
:103E2D000FEEB409EE9002C4122954642D70600F88
:103E3D009002C7F09002C4122954FE642E60051240
:103E4D002A5680F07F069002617430F0A3DFFC905B
:103E5D000261742DF09002C7E024FE60131460150A
:103E6D001460171460192404701A9002C8023E944D
:103E7D00122AC68012122A6D800D122A288008126D
:103E8D0029C580031229E9E0900266F0023EFCE4A8
:103E9D009002C7F09002C4122954FE642E600512E0
:103EAD002A5680F07F069002617430F0A3DFFC90FB
:103EBD0002C7E024FE601314601614601814601A13
:103ECD002404701B9002C8023EF7122AC6023EF768
:103EDD00122A6D8015122A2880101229C5800B9088
:103EED0002C8E0900261F01229E9E0900266F0E468
:043EFD00900267F0D8
:013F0100229D
:065D9C009002F1122A44FE
:105DA200E4FFFE9002F11229546009B42C010E0F97
:105DB200EEB402EF9002F1122954B441037F0122A2
:025DC2007F0060
:015DC40022BC
:063C33009002F4122A4485
:103C3900E4FFFE1229516009B42C010E0FEEB40302
:103C4900F2E4FE122951FD642E600C74812E1229B2
:103C590048EDF00E0F80EC9002F412298574812E44
:103C6900122948EDF00E0F12295CFD74812E1229DC
:103C790048EDF00E0F12295CFD74812E122948EDD2
:103C8900F00E0F122951642C60030F80F61229508F
:103C9900FD74812E122948EDF00E0F74812E122920
:103CA90048742FF00E122951642C60030F80F60F0F
:103CB900122951FD642E600C74812E122948EDF0F1
:103CC9000E0F80EC9002F412298574812E12294876
:103CD900EDF00E0F12295CFD74812E122948EDF0CA
:103CE9000E0F12295CFD74812E122948EDF00E0F7A
:103CF900122951642C60030F80F6122950FD74813A
:103D09002E122948EDF00E74812E122948E4F07F15
:0E3D1900997E011260A6BF010312142C7F01D7
:013D27002279
:10142C00900281122A4DA3E024D02F90029FF090BD
:10143C0002847D6412296C9002831229A990028681
:10144C00122964EF2BFFEE3AFEA3E09002971229CB
:10145C0099900288E09002A1F0E49002A3F090022F
:10146C00A3122945E0642F600512297B80F0122914
:10147C007BE4FF9002A3122945E0642E600612293A
:10148C007B0F80EFEF24FB603504707590028A129D
:10149C002A4DA3E024D02F9002A0F090028D7C0066
:1014AC007D641229B1AA06AB0790028C1229AD906B
:1014BC00028F12296412298E900291021508900253
:1014CC008B122A4D90028AE090028C122AAC900268
:1014DC00A0F090028EE024D0FFE434FFFE7C007D6F
:1014EC006412036990028D1229A9EF2BFBEE3AFAD4
:1014FC0090029012296A12298E900292E09002A218
:10150C00F07F9B7E011260A690029BE4F0A3EFF0AB
:10151C007F9A7E011260A6BF0130122A9A9002981F
:10152C00E02FF0900297E03EF0C3A3E0947090029D
:10153C0097E09417404BA3E02490F0900297E0348E
:10154C00E8F090029FE004F08037122A9A900297FC
:10155C00122AD24008900297122ADC80249002981A
:10156C00E02470F0900297E03417F0122A9AC3909E
:10157C000298E09FF0900297E09EF090029FE0149A
:10158C00F07F9D7E011260A690029DE4F0A3EFF027
:10159C007F9C7E011260A6BF0130122AA390029A92
:1015AC00E02FF0900299E03EF0C3A3E0947090021B
:1015BC0099E09417404BA3E02490F0900299E0340A
:1015CC00E8F09002A0E004F08037122AA390029970
:1015DC00122AD24008900299122ADC802490029A96
:1015EC00E02470F0900299E03417F0122AA3C39013
:1015FC00029AE09FF0900299E09EF09002A0E01415
:10160C00F0E49002A3F090029F122AB9122945EE41
:10161C0012297A122A81FF122945122979900297F0
:10162C001228F5742E12297A900297122A0D900224
:10163C00A31229451229797C007D0AAF03AE021250
:10164C002A201229451229799002A1E0FF9002A3C9
:10165C00122933742F12297A9002A0E0FFD39463DD
:10166C00401EE0FE75F064842430FD9002A3122924
:10167C0045ED12297AEE75F00A84122A82FE800654
:10168C009002A0122AB9122945EE12297A122A8147
:10169C00FF1229451229799002991228F5742E12FD
:1016AC00297A900299122A0D9002A3122945122927
:1016BC00797C007D0AAF03AE02122A201229451252
:0F16CC0029799002A2E0FFA3122933E412297AB0
:0116DB0022EC
:1043E400900268E0F97002FF22900294E0FEA3E0DC
:1043F400FF90025FE0FAA3E0FBD39FEA9E4008EB44
:104404009FFDEA9EFC801590025FE0FEA3E0FFC3DF
:10441400900295E09FFD900294E09EFCD3ED94B44D
:10442400EC9400401074689D9002FCF074019C9020
:1044340002FBF080089002FBECF0A3EDF0D39002B5
:10444400FCE094199002FBE094004006E490027EA4
:10445400803A90027EE004F0E9C3940A500CE0C371
:1044640094324003E480257F0022900268E0C394E4
:1044740032500F90027EE0C3941E4003E4800D7F0F
:10448400002290027EE0C394144014E4F090025F92
:10449400E0FFA3E0900294CFF0A3EFF07F01227F2E
:0144A4000017
:0144A50022F4
:063858009002D6122A4482
:10385E00E4FCFD1229828C8212295E6009B42C01CF
:10386E000D0CEDB407ED1229828C8212295EB42C58
:10387E0003E48041E4FD1229828C8212295EFF64EA
:10388E002E6005122A8B80EEED24FD601004701F51
:10389E009002D9122A4DA3E024D02F80189002DA7C
:1038AE00122A4D9002D9E09002DB122AAC800690CB
:1038BE0002D9E024D0900268F01229828C8212295B
:1038CE005E642C60030C80F10C1229828C8212290A
:1038DE005EB42C08E490025FF0A3F022E4FD1229FE
:1038EE00828C8212295EFF642E6005122A8B80EE76
:1038FE00ED24FD600C0470389002D912296AA38061
:10390E001B9002DA12296AAA06AB079002D97D64CF
:10391E0012296EEF2BFFEE3AFE9002DBE024D0FD73
:10392E00EC34FFCD2FFFED3E90025FF0A3EFF022BF
:10393E009002D9E024D0FEE434FF90025FF0A3CED3
:01394E00F088
:01394F002255
:10598600900207122A4490020A122985120301FF87
:1059960060259002071229851203016F60037F00BC
:1059A60022900208E475F0011203D090020BE47510
:0A59B600F0011203D080CF7F012220
:105F1100A3E02403F582E43401F583E59BF09001CD
:105F210085E004F022E02403F582E43401F583E402
:025F3100F0225C
:0300430002475C15
:10475C00C0E0C0F0C083C082C0D075D000C000C023
:10476C0001C002C003C004C005C006C007E59A30F2
:10477C00E106539AFD0247D7E59A30E04E539AFE74
:10478C00900184E064017015125F11E59BB40A0B73
:10479C00125F26125F1F125DEE802B802490018425
:1047AC00E064037021125F11900102E004F0E59BBC
:1047BC00B40A0E900185125F26125F1F12561580E7
:1047CC00051262298005900185E4F0D007D006D04F
:1047DC0005D004D003D002D001D000D0D0D082D0EC
:0647EC0083D0F0D0E032A2
:0C622900900185E0D3947E4002E4F02256
:0D620400E4F5A2759A50758E10759CF42279
:10097B004750532000B1B1CEB33A2000C4CFCEB311
:10098B003A2000B6ABBEAD3A2000CEF7BEAD3A2052
:10099B0000BAA3B0CE3A2000202020475731303088
:1009AB003020202000535441545553204F4B2100ED
:1009BB002020C6F8CFF3BDD3BFDAB0E5202000204E
:1009CB00202020C3BBC1ACBDD3A3A1202000576501
:1009DB0061746865722053746174696F6E004E6F39
:1009EB0020636F6E6E656374696F6E2120005765AF
:1009FB00617468657200504D32353A2030303000EA
:100A0B0025007061004449523A005753203A002F99
:100A1B0000204D2F5300524E203A006D6D00504F69
:100A2B00533A00202020004D53473A00416E74008A
:100A3B005758004469676900436172000000180051
:100A4B00240024F4190C0204040004000400040024
:100A5B000204010800F0000000000000000000008C
:100A6B00000000002020202020002000505000001B
:100A7B00000000005050F850F850500010385070E3
:100A8B0028287000006868102058580030283070F3
:100A9B0048483000101000000000000010202020FB
:100AAB00202010002010101010102000002070705B
:100ABB0070200000002020702020000000000000AB
:100ACB000010100000000078000000000000000083
:100ADB000000200008081010202040003048484833
:100AEB00484830002060202020207000304808103B
:100AFB002040780030480830084830001030305023
:100B0B0050781000784040700808700030484070F2
:100B1B0048483000784808102020200030484830E2
:100B2B004848300030484838084830000000200062
:100B3B000020000000002000002040000810204092
:100B4B0020100800000078007800000040201008FA
:100B5B001020400030480810200020003048485832
:100B6B002828380030484848784848007048487072
:100B7B004848700030484040404830007048484872
:100B8B004848700078404070404078007840407092
:100B9B00404040003048405848483000484848786A
:100BAB0048484800702020202020700008080808C2
:100BBB00484830004848506050484800404040404A
:100BCB00404078004878784848484800486868585A
:100BDB00584848007848484848487800704848705A
:100BEB0040404000304848486858380070484870CA
:100BFB0060504800304840300848300078202020B2
:100C0B002020200048484848484830004848484879
:100C1B0030303000484848487878480048483030F1
:100C2B003048480088885020202020007808103059
:100C3B002040780030202020202030008080404051
:100C4B002020100030101010101030002050000029
:100C5B0000000000000000000000780020200000D1
:100C6B000000000000000038384838004040407059
:100C7B004848700000000038404038000808083829
:100C8B0048483800000000307840300000102078D1
:100C9B0020202000000000384838083040404070C9
:100CAB0050505000000020002020200000001000B9
:100CBB001010106040404058605048002020202009
:100CCB002020700000000078585858000000007079
:100CDB0048484800000000304848300000000070D1
:100CEB004848704000000038484838080000005859
:100CFB006040400000000038601870000000207059
:100D0B002020300000000048484838000000004810
:100D1B0048303000000000A8A870500000000048C8
:100D2B003030480000000048483808300000007898
:100D3B001020780030202040202030002020202060
:100D4B002020200060202010202060002850000070
:0C0D5B000000000000707070707000005C
:100D670090022BE0FBA3E0FAA3E0F9900231E0F553
:100D77008275830012031AFF90022FE02433F58255
:100D8700E43402F583EFF090022FE004F090023193
:100D9700E004F0900230E004F0E02290022FE0241B
:100DA70033F582E43402F583E4F0900234E024D092
:100DB700FFE434FFFE7C007D0A120369AA06AB0735
:100DC700900233E024D0FFE434FFFE7D6412036910
:100DD700EF2BFFEE3AFE900235E024D0FDEC34FF16
:100DE700CD2FFFED3EFEE4FD90023D120522E47F8C
:100DF700FEFEFDFC90023DE0F8A3E0F9A3E0FAA3B4
:100E0700E0FB1203E6E47BE87A03F9F81204719039
:100E17000241120522900241A3A3E0FFA3E0900242
:100E270039CFF0A3EFF0900239E0FAA3E0FB7C00A2
:100E37007D64FFAE0212037B7C007D0A12037BED0B
:100E47002430900233F0AF037C007D0AAE02120318
:100E57007B7C007D0A12037BED243022E02411F510
:100E670082E43402F583EEF090020DE004F0EF75B2
:100E7700F00A8475F00A84E5F02430FEE02411F5C9
:100E870082E43402F583EEF090020DE004F0EF7592
:100E9700F00A84E5F02430FEE02411F582E4340200
:100EA700F583EEF090020DE004F02290022FE0248B
:100EB70033F582E43402F583E4F0900234E024D081
:100EC700FFE434FFFE7C007D0A120369AA06AB0724
:100ED700900233E024D0FFE434FFFE7D64120369FF
:100EE700EF2BFFEE3AFE900235E024D0FDEC34FF05
:100EF700CD2FFFED3EFE900239F0A3EFF022E02464
:100F0700A6F582E43402F583EFF09002A5E004F041
:100F1700E024A6F582E43402F58322900247E0FB41
:100F2700A3E0FAA3E0F902030174002DF582E4348B
:100F370000F583E0FF900210E02416F582E4340206
:100F4700F5832290022BFFF0900225E475F0010251
:100F570003D090024DE0FEA3E02467F582740A3EB9
:100F6700F583E49322EFF0A3EDF0A3EBF0A3EAF00F
:100F7700A3E9F02224E0FFE434FFFEEF780322FD2B
:100F8700900232E02433F582E43402F583229002A2
:100F970031F0E4900230F02290024BE004F0E004DC
:100FA700F090024AE004F022900228E004F0E00406
:100FB700F0900227E004F022EFF0900210E004F036
:100FC70022EFF09002A5E0042290022FE02433F5EF
:100FD70082E43402F583E4F022900232E004F0E088
:100FE70004F0900231E004F0227DA11203690C7D28
:100FF7006812037BA3EEF0A3EFF022FF90024BE011
:10100700244FF582E43402F583EFF090024EE004BA
:10101700F022FF900228E0242DF582E43402F583C4
:10102700EFF090022CE004F022A3F0900239E0FEEA
:10103700A3E0FF2274812FF582E43402F583E0FFF9
:101047009002A522900234F07C007D0AAF03AE0225
:101057002290023B7D0AE0FAA3E0FB7C00FF22FF1F
:10106700E433FE90020FE0FDC39FEE6480F87480C6
:1010770098227420F090023BE0FEA3E0FF22F0905C
:10108700020FE004F02290024DFFEEF0A3EFF022F2
:10109700E490024BF090024AF022E4900228F0908C
:1010A7000227F022E49002A5F09002A422F07B012F
:1010B7007A02791622EF25E0FF0EEE22F09002A4C5
:1010C700E004F022900235F0E4A3F0900233E0222E
:1010D7009002A4E0FFC322E4900232F0900231F0C4
:0110E70022E6
:102AE6007F337E001260A6EF64016003022C937FA1
:102AF6008D7E011260A6EF7003022C937F30124D7B
:102B0600CD7F01124DCD7F0A7E00125FC77F061270
:102B16004DCD7F0C124DCD1256FC7BFF7A09797B89
:102B2600E4FD7F011251BEE49002A5F090025F7DA4
:102B36006412105DAE0212037BEF2430FF9002A5F3
:102B4600120F17120FC8120E4CFF120F17120FC8D2
:102B5600F090025FE0FEA3E0FF120E58FF9002A580
:102B6600120F057420120F10E4F07D03122C9490BE
:102B76000268E0FF7E007C007DB91203697D641265
:102B8600037BAB07AA06E49002A5F0FC7D64120E57
:102B960055FF120F17120FC8120E4CFF120F171205
:102BA6000FC8F0AE02AF03120E58FF120F05744B9A
:102BB600120F10746D120F10E4F07D05122C947B29
:102BC6000E7D08E4FF125402900288E07BFFB44EAB
:102BD600067A09798080047A097987E4FD7F0212F2
:102BE60051BE1210ABF01210D79407500E12103BC4
:102BF600120F17120FC81210C380EB9002A5120F06
:102C060017E4F07F02122CA0900292E07BFFB445FD
:102C1600067A09798E80047A097995E4FD7F031294
:102C260051BE1210AB7409F01210D79411500E1247
:102C3600103B120F17120FC81210C380EB9002A59B
:102C4600120F17E4F07F03122CA07BFF7A09799C00
:102C5600E4FD7F041251BE1210ABF01210D7940699
:102C6600501674612FF582E43402121043120F17C6
:102C7600120FC81210C380E39002A5120F17E4F0DA
:0D2C86007B017A0279A67D037F041251BE06
:102C9300227B017A0279A67F011251BE227B017A3F
:092CA3000279A67D031251BE2244
:103950007F337E001260A6EF64016003023A4612D4
:103960005DC57F01124DCD7F0A7E00125FC77BFFD0
:103970007A0979A37F011255C17BFF7A6079297F8B
:10398000021255C1E490020EF090020EE0FFC394C3
:1039900010501474112FF582E43402F583E4F09092
:1039A000020EE004F080E290020FE4F0A37410F045
:1039B000FF7E001260A6E490020DF0EF75F06484C3
:1039C0002430FE120E63900210E004F070069002A4
:1039D0000FE004F0E490020EF090020DE02411F5E7
:1039E00082E43402F583742E120EAA90020FE0FED8
:1039F000A3E0FF1260A6EF75F064842430FE90020D
:103A00000D120E63900210E004F0700690020FE0B9
:103A100004F090020EE004F0E0C3940340BB1247B0
:103A2000F27B017A0279CE7D067F021251BE7B01C4
:103A30007A0279117F041255C17BFF7A0979B07D32
:063A4000017F031251BEDC
:013A4600225D
:0910E80090022B120F72A3EDF02F
:1010F1007F337E001260A6EF640160030213CE7F8E
:101101000B7E011260A6EF70030213CE7F30124DE9
:10111100CD7F01124DCD7F0A7E00125FC77F06127F
:101121004DCD7F0C124DCD1256FC90022EE0702B4E
:101131007BFF7A0979BBFD7F011251BE7BFF7A09E2
:1011410079CA7F0212141B7A0979D97F0312141B01
:101151007A0979E9E4FD7F040251BE7A0979F97FC0
:10116100011213E3740D120F98120D67B403FA12F2
:101171000EB2C39420EE94005015121032C37420A5
:101181009FF0E49E900239F0E4900232F0801490D6
:10119100023AE024E0F0900239E034FFF0900232AC
:1011A1007401F01210327C007D0A1203697D121263
:1011B1000FF8900232E07006A3742DF080069002C1
:1011C100337420F012107CC3940AEE9400500C90FA
:1011D10002347420F07C007D0A800F90023BE0FA1B
:1011E100A3E0FBFF120E4F12104B120E5CA3F0E4B2
:1011F100A3F07F011214057A0A7947E4FD7F0712F3
:1012010054BC7B0E7D08E4FF1254027A0A79017FF7
:10121100021213E37419120F98120D67B402FA1235
:101221000FD07B017A0279337D067F021251BE7B9A
:10123100FF7A0A790B7D077F021251BEE490022FDB
:10124100F0741C120F95120D67B404FA120FD090AE
:101251000233E0B430037420F07F031214057A0ADC
:10126100790D7D077F031251BE1247F27B017A028D
:1012710079CEE4FD7F0912142304120F95120D6734
:10128100B403FA120FD0900233E0B4300B7420F0A3
:10129100A3E0B430037420F07A0A79107D081214A7
:1012A100137D081213CF7405120F98120D67B40342
:1012B100FA120EB2120FF09002337420F0C3EF94C1
:1012C1000AEE9400500CA3121079120E58900235B8
:1012D100800D121058120E5312104B120E5CA3F017
:1012E100E4A3F07A0A79157D101214137D101213FC
:1012F100CF7409120F98120D67B403FA120EB212CD
:101301000FF0C3940AEE9400500E9002331210793C
:10131100120E589002348010121058120E5390027F
:101321003312104E120E5CA3F0E4A3F07D101213E1
:10133100F37D107F0D12362F7BFF7A0A791C7D1009
:101341007F0E1214239002317411120F98120D673F
:10135100B403FA120DA2121030120E581210CBB4AF
:10136100300B7420F0A3E0B430037420F07BFF7ADB
:101371000A79217D187F0812362F7B017A02793391
:101381007D187F0A12362FE490022FF090023174FB
:1013910015120F98120D67B403FA120DA212103034
:1013A100120E581210CBB4300B7420F0A3E0B430FD
:1013B100037420F07D181213F37D187F0D12362F60
:0D13C1007BFF7A0A79267D187F0F12362FE8
:1013CE00227B017A0279337F0A12362FE490022FA4
:1013DE00F0900231227BFFE4FD1251BEE490022F09
:1013EE00F0900231227BFF7A0A791A7F0C12362F87
:1013FE007B017A027933227B017A0279337D0512E1
:10140E0051BE7BFF227BFF7F0812362F22E4FD1296
:0E141E0051BE7BFF2212362FE490022FF022E7
:101BFB007F337E001260A6EF64016003021E477FF5
:101C0B008B7E011260A6EF7003021E477F30124DD0
:101C1B00CD7F01124DCD7F0A7E00125FC77F06126A
:101C2B004DCD7F0C124DCD1256FC9002157408F061
:101C3B002408FD7BFF7A0A7929E4FF12362F9002E4
:101C4B0015E02410FD7BFF7A0A792EE4FF12362F64
:101C5B00E4FB7D107F081254027BFF7A0A79327DF8
:101C6B00027F08123145E490020FF090020FE0FF63
:101C7B00C3940C500C74162F120F42E41210858073
:101C8B00EAE4900210F090020F7407F090020FE05C
:101C9B00FFC3940D502074002FF582E43400F583BC
:101CAB00E0C313900211F064206006120F3A120F7A
:101CBB00BF12108680D690000DE0541EC313900205
:101CCB0011F0D39400403C120F3C742D120FC0A3A3
:101CDB00E0FFC3940A5009EF2430FF900210801DDF
:101CEB00900211E0FF75F00A842430FE120F3CEED7
:101CFB00120FC0EF75F00A84E5F02430FF120F3F8E
:101D0B00120FBF120F3CE41210B47F011255C19099
:101D1B000212740DF0E4A3F0900213E0C39406409A
:101D2B0003021E47900212E0FF2400F582E4340008
:101D3B00F583E020E003021E3BE4900210F0120F4B
:101D4B003F7420120FC0EF240490020FF090021288
:101D5B00E0240C121066500B120F30120FBF121032
:101D6B008680EA120F3CE4F0900215E02408FD1285
:101D7B0010B57F0312362FE4900210F0900212E0A0
:101D8B00240D90020FF0900212E0241612106650F0
:101D9B000B120F30120FBF12108680EA120F3CE4A9
:101DAB00F0900215E02410FD1210B57F0312362FB0
:101DBB00900212E02416F582E43400F583E09002E1
:101DCB0014F024DD601C24E5602024DF600C24ED7E
:101DDB0070207BFF7A0A793780257BFF7A0A793B63
:101DEB00801D7BFF7A0A793E80157BFF7A0A794347
:101DFB00800D900214E0900216F0E4A31210B47D53
:101E0B00067F011251BE900212E02417F0E0FF9002
:101E1B000100E0C39FFE900210F074002FF9E43430
:101E2B0000FA7B01900227EEF07D027F0A0240C090
:0C1E3B00900212E02407121085021D2303
:011E47002278
:0755C100900222EF120F70AF
:1055C8007F30124DCD900222E024FE600E14600F51
:1055D800146010240370117F80800A7F9080067FFA
:1055E8008880027F98124DCDE4900226F090022325
:1055F800120F25FF6016124E47900224120F529088
:0C5608000226E004F0E0D3941040E222FF
:015614002273
:0651BE00900245120F6C87
:1051C4007F30124DCD900245E024FE60121460172A
:1051D40014601C24037022900246E0248080169000
:1051E4000246E02490800E900246E02488800690D7
:1051F4000246E02498FF124DCDE490024AF090025A
:1052040047120F25FF6016124E47900248120F52A4
:0D52140090024AE004F0E0D3941040E22242
:01522100226A
:0654BC00900245120F6C86
:1054C200E4A3F07F34124DCD900246E02480FF1217
:1054D2004DCD900245E02480FF124DCD7F30124D1C
:1054E200CD900247120F25FF124E47900248120F2D
:1054F20052900247120F25FF124E47900248120F98
:1055020052900246E004F090024AE004F0E0C394B4
:035512001040B096
:015515002273
:0A540200900246EBF0900245EFF037
:10540C00C3ED9F900248F0E4900247F0900248E010
:10541C00FF900247E0C39F50367F34124DCD90026F
:10542C0046E02480FF124DCD900245E02480FF120F
:10543C004DCD7F30124DCD7FFF124E477FFF124E68
:10544C0047900245E004F0900247E004F080BD7FF5
:04545C0036024DCDFA
:06362F00900245120F6C31
:10363500120F2270030236F9900246E090024CF018
:10364500E490024AF090024AE0FFC39410501074CF
:103655004F2FF582E43402F583E4120FA780E612BA
:103665000F22120F7BC333CE33CED8F912108D1231
:103675001097120F59121002700690024DE004F0D7
:10368500120F9FE0B408EB900248120F52120F225E
:1036950070131210981236FEA3120FA5E0C39408FA
:1036A50040F30236F9120F22120F7BC333CE33CE0D
:1036B500D8F912108D90024B7401F0E490024AF093
:1036C500120F59121002700690024DE004F0120F0D
:1036D5009FE0B408EB1210971236FEA3120FA5E077
:1036E500C3940840F3900248120F52900245E0043B
:0936F500F00236357F36024DCD9E
:1036FE007F34124DCD90024CE02480FF124DCD90C0
:10370E000245E02480FF124DCD7F30124DCD900248
:10371E004BE0244FF582E43402F583E0FF124E476E
:10372E0090024BE004F0E0244FF582E43402F5837E
:0C373E00E0FF124E4790024BE004F02226
:0640C000900222120F6CB9
:1040C600A3E07003024194900227E0FFC31390021D
:1040D60029F0EF5401A3F0E4900228F0900229E0C1
:1040E600FF900228E0C39F506E900224120F251203
:1040F6000F4AEF640D700302419490022BE0FE64B8
:104106000A7003024194900224120F2590022C1289
:104116000F4DBF0D0690022C7420F090022CE0B4D7
:104126000A037420F0900222E0FFA3E0FDAB0690A4
:10413600022CE0900230F0124321900222E004F0BB
:10414600E0D3940F40087408F0A3E02408F090022E
:1041560028E004F00240E290022AE0602C9002245B
:10416600120F25120F4AEF640D602390022BE0FB1D
:10417600640A601AE490022CF0900222E0FFA3E0A9
:0E418600FDE4900230F01243217F36124DCD41
:014194002208
:0843210090022DEFF0A3EDF076
:10432900E4900231F0900231E0FFC39410500C7414
:10433900332F120F8DE4120FE880EAEB120F7BC3C3
:1043490033CE33CED8F9FF1210DE74672F120F6205
:10435900120F86EDF00FBF00010E120FE0E0B40856
:10436900E9900230E0FD602D120F7BC333CE33CECE
:10437900D8F9FF9002327401F0E4900231F07467C9
:104389002F120F62120F86EDF00FBF00010E120FF0
:10439900E0E0B408E91210DE7F34124DCD90022E10
:1043A900E02480FF124DCD90022DE02480FF124DB4
:1043B900CD7F30124DCD120F871243D8120F8A12BA
:0E43C90043D890022E120FE6E0C3940840CABB
:0D43D70022E0FF124E47900232E004F02277
:0E314500900224120F72900222EFF0A3EDF020
:10315300900229EFF0A3EDF0900224120F257003E3
:10316300023255E4900227F0900227E0FFC3941047
:103173005010742D2FF582E43402F583E4120FB757
:1031830080E6900224120F25120F7BC333CE33CE79
:10319300D8F990022B1210901210A190022B120F4B
:1031A3005C121019700690022BE004F0120FAFE0CE
:1031B300B408E8900225120F52900224120F2570D2
:1031C300151210A212325A90022A120FB5E0C394BC
:1031D3000840F1023255900224120F25120F7BC3CF
:1031E30033CE33CED8F9FF90022BEEF0A3EFF0905D
:1031F30002287401F0E4900227F090022B120F5C76
:10320300121019700690022BE004F0120FAFE0B415
:1032130008E81210A112325A90022A120FB5E0C325
:10322300940840F1900222E004F0900225120F521C
:10323300900222E0D3940F400E7408F090022AE02B
:10324300900223F002315B900223E090022AF00205
:07325300315B7F36024DCD17
:10325A007F34124DCD90022AE02480FF124DCD908A
:10326A000222E02480FF124DCD7F30124DCD900214
:10327A0028E0242DF582E43402F583E0FF124E475C
:10328A00900228E004F0E0242DF582E43402F5836C
:0C329A00E0FF124E47900228E004F022F2
:105DC5007F30124DCD7F01125DE37F06125DE37FCB
:105DD5000C124DCD7F0A7E00125FC70256FC124D94
:095DE500CD7F0A7E00125FC72287
:1056FC00E4900246F0E4900245F07F34124DCD90D8
:10570C000246E02480FF124DCD900245E02480FF3C
:10571C00124DCD7F30124DCDE4FF124E47E4FF12F7
:10572C004E47900245E004F0E0C3941040CC900248
:0A573C0046E004F0E0C3942040BBF7
:015746002240
:104DCD00D2C1E4FEC2C500D2C5000EEEB405F5C2D7
:104DDD00C1C2C1C2C500D2C500C2C1C2C500D2C5C3
:104DED0000C2C1C2C500D2C500E4FEEF30E704D257
:104DFD00C18002C2C1C2C500D2C5001210BCB4042C
:104E0D00EAC2C1E4FEC2C500D2C5000EEEB404F57F
:104E1D00E4FEEF30E704D2C18002C2C1C2C500D2A8
:104E2D00C5001210BCB404EAC2C1E4FEC2C500D272
:0A4E3D00C5000EEEB404F502614753
:104E4700D2C1E4FEC2C500D2C5000EEEB405F5C25C
:104E5700C1C2C1C2C500D2C500D2C1C2C500D2C538
:104E670000C2C1C2C500D2C500E4FEEF30E704D2DC
:104E7700C18002C2C1C2C500D2C5001210BCB404B1
:104E8700EAC2C1E4FEC2C500D2C5000EEEB404F505
:104E9700E4FEEF30E704D2C18002C2C1C2C500D22E
:104EA700C5001210BCB404EAC2C1E4FEC2C500D2F8
:0A4EB700C5000EEEB404F5026147D9
:105FC700EF1FAC0670011E4C6010E4F5D875F9FCA4
:0B5FD70075E966D2DE20DFE880FB22C7
:10614700E4FF000000000000000000000FEFB46E45
:01615700F156
:016158002224
:10004600EC4D6011E8497017ED33EC3304600DE4B4
:10005600FCFFFEFD22E933E8330470F80201F612D4
:1000660001C158046009E4CC2481500628500902D5
:1000760002002840030201FDC0E0EB4A7044B9804B
:1000860006D0E0FB0201ECEF4E701CBD8008EBFFD2
:10009600EAFEE9FD80EBE98DF0A4FEE5F002012F12
:1000A600E9CDF9EAFEEBFFEF89F0A4FCE5F0CE8995
:1000B600F0A42EFFE435F0CD89F0A42DFEE435F052
:1000C6008067EF4E7005BD80D780C3EF8BF0A4AC80
:1000D600F0EE8BF0A42CFCE435F0F8EF8AF0A42CBB
:1000E600E5F038FCE433CB8DF0A42CFCE5F03BF8CE
:1000F600EE8AF0A42CFCE5F038F8E433CF89F0A4BE
:100106002CFCE5F038CF3400CE89F0A42FFFE5F0C3
:100116003EFEE433C98DF0A42EFEE5F039CD8AF01B
:10012600A42FFFE5F03EFEE43DFD33D0E0FB500793
:100136000BBB000F020200EC2CFCEF33FFEE33FE8C
:06014600ED33FD0201D8BB
:10014C0075F020800E75F010800575F0087D007E2E
:10015C00007F003392D530D503120503EC334010E9
:10016C00EF33FFEE33FEED33FDEC33FCD5F0ED2237
:0E017C00E5F0247EA2D513CC92E7CDCEFF2273
:10018A00EDD2E7CD33EC3392D524814006E4FFFE6D
:10019A00FDFC22FCE4CFCECDCC24E0501174FF80CC
:1001AA00EDC3CC13CCCD13CDCE13CECF13CF047069
:0701BA00F030D5DE02050361
:1001C100E9D2E7C933E833F892D5EDD2E7CD33EC84
:0701D10033FC5002B2D522FD
:1001D800EC30E7100FBF000C0EBE00080DBD000488
:1001E8000BEB6014A2D5EB13FCED92E7FD2274FF34
:1001F800FCFDFEFF22E480F8A2D574FF13FC7D808D
:03020800E480EFA0
:0300000002623564
:0C623500787FE4F6D8FD7581220260BD80
:10020B00E709F608DFFA8046E709F208DFFA803ED5
:10021B0088828C83E709F0A3DFFA8032E309F608C2
:10022B00DFFA8078E309F208DFFA807088828C832A
:10023B00E309F0A3DFFA806489828A83E0A3F608DE
:10024B00DFFA805889828A83E0A3F208DFFA804CB8
:10025B0080D280FA80C680D4806980F2803380108F
:10026B0080A680EA809A80A880DA80E280CA8033F8
:10027B0089828A83ECFAE493A3C8C582C8CCC58370
:10028B00CCF0A3C8C582C8CCC583CCDFE9DEE78040
:10029B000D89828A83E493A3F608DFF9ECFAA9F0BF
:1002AB00EDFB2289828A83ECFAE0A3C8C582C8CC15
:1002BB00C583CCF0A3C8C582C8CCC583CCDFEADE2E
:1002CB00E880DB89828A83E493A3F208DFF980CC90
:1002DB0088F0EF60010E4E60C388F0ED2402B40489
:1002EB000050B9F582EB2402B4040050AF23234530
:0602FB00822390025B73F8
:10030100BB010689828A83E0225002E722BBFE02FA
:09031100E32289828A83E493222D
:10031A00BB010CE58229F582E5833AF583E0225098
:10032A0006E92582F8E622BBFE06E92582F8E222E2
:0D033A00E58229F582E5833AF583E49322FC
:10034700F8BB010DE58229F582E5833AF583E8F0EC
:10035700225006E92582C8F622BBFE05E92582C898
:02036700F22280
:10036900EF8DF0A4A8F0CF8CF0A428CE8DF0A42EA8
:02037900FE2262
:10037B00BC000BBE0029EF8DF084FFADF022E4CC66
:10038B00F875F008EF2FFFEE33FEEC33FCEE9DEC2F
:10039B00984005FCEE9DFE0FD5F0E9E4CEFD22ED75
:1003AB00F8F5F0EE8420D21CFEADF075F008EF2FBF
:1003BB00FFED33FD4007985006D5F0F222C398FDB0
:0503CB000FD5F0EA224D
:1003D000C5F0F8A3E028F0C5F0F8E58215827002B8
:0603E0001583E038F02255
:1003E600E88FF0A4CC8BF0A42CFCE98EF0A42CFCB6
:1003F6008AF0EDA42CFCEA8EF0A4CDA8F08BF0A434
:100406002DCC3825F0FDE98FF0A42CCD35F0FCEB92
:100416008EF0A4FEA9F0EB8FF0A4CFC5F02ECD3957
:0F042600FEE43CFCEAA42DCE35F0FDE43CFC22C4
:1004350075F008758200EF2FFFEE33FECD33CDCC7E
:1004450033CCC58233C5829BED9AEC99E582984001
:100455000CF582EE9BFEED9AFDEC99FC0FD5F0D6DE
:10046500E4CEFBE4CDFAE4CCF9A88222B800C1B908
:100475000059BA002DEC8BF084CFCECDFCE5F0CB46
:10048500F97818EF2FFFEE33FEED33FDEC33FCEB7F
:1004950033FB10D703994004EB99FB0FD8E5E4F93A
:1004A500FA227818EF2FFFEE33FEED33FDEC33FC27
:1004B500C933C910D7059BE99A4007EC9BFCE99A1B
:1004C500F90FD8E0E4C9FAE4CCFB2275F010EF2F60
:1004D500FFEE33FEED33FDCC33CCC833C810D70760
:1004E5009BEC9AE899400AED9BFDEC9AFCE899F89B
:0E04F5000FD5F0DAE4CDFBE4CCFAE4C8F9222E
:0E050300C3E49FFFE49EFEE49DFDE49CFC2209
:10051100EB9FF5F0EA9E42F0E99D42F0E89C45F040
:0105210022B7
:0C052200ECF0A3EDF0A3EEF0A3EFF0224C
:00000001FF
